:020000041100E9
:10300000002310B5294C0120636101F003FA402030
:103010000223FE21264A207401F082FA002835D1CD
:103020000223FF21234A207C01F07AFA00282DD1C7
:10303000214BA2899A4226D1E389204A93420ED19C
:103040001F4B204963612368002B05D1002903D061
:103050000C22200008F004FB01F050FA10BD1A4ABF
:10306000934201D00021EEE7184B194A1B689342A6
:1030700005D9C0220421207C920001F0CBFA104B2C
:1030800014496361DFE700232374EBE7CC22382087
:10309000AC219201207401F0BDFA0028F3D10E4B4F
:1030A0000E4963610E4BE381CDE7C046E862FF1F26
:1030B000F462FF1FF662FF1F5959000083050000EC
:1030C00079420011D4BB0011821500002C63FF1F50
:1030D00087130000E0BB001115430011C8BB0011AD
:1030E000AAAAFFFFF7B5164B0192C318021D0020D4
:1030F000009388235B05D3181B685C1C1AD09CB214
:10310000402C18D88D781E0CAC466746CD782D0221
:103110003D43AE4206D1019800280ED110000C703C
:10312000240A4C7003249BB20733A343D218009B9C
:103130009A42DED3FEBD4432F9E71000FAE7C046FA
:10314000FC0F0000802213B503000324019189B213
:10315000520107319B18A14304305A1A88235B059A
:10316000C3181B68591C03D190429241104016BDF0
:1031700099B2402907D80B000733A343C0189042E7
:10318000ECD30020F3E74430F9E7134B134A1B68F4
:10319000126810B5FA24934201D81A00F824104B93
:1031A000E4021B689A4210D813000E4A12689A4231
:1031B0000ED3013307D1F823DB029C4203D10A4925
:1031C000054808F01DFB200010BDFC24E402ECE7DC
:1031D000FE24E402F7E7C04600C0071100D0071143
:1031E00000E0071100F00711FFFFFF7FF0B59BB073
:1031F000150004900391402A00D9A0E006AB598045
:103200001A80FFF7C2FF0400042816D9002206A97D
:10321000FFF768FF052810D906AB1B88AB420CD11D
:10322000002D07D0514B2A000499C01808F048FC23
:10323000002802D101201BB0F0BD06AB1D8020008C
:103240000699FFF77FFF041E7BD1069B0793FFF7CC
:103250009CFF80235B01C618802307001B039E424E
:1032600001D3F826F60288235B05F31801931B6847
:10327000013302D0019808F033FC3D49019808F071
:10328000BFFA3B1D0293331D05938822029B520512
:103290009B181B6808935A1C3CD044219AB2009199
:1032A000402A04D80320D11D814389B2009103999B
:1032B0001B0C8B4224D0402A22D80122300008A9BE
:1032C000FFF710FF021E1BD1380008A9FFF70AFF05
:1032D0000400042831D9009A059B9B1880225201D2
:1032E000B218934240D288235B05C118009A09A8FE
:1032F00008F036F91D4B009A09A9F01808F008F9F2
:10330000009A029B9446634402931A4B029AFB185C
:103310009A42BAD388235B05FC18216801980139C9
:1033200008F06EFA200008F0DBFB039A07AB5A8026
:1033300030000799FFF706FF0400002C03D100209E
:1033400079E70428FBD988235B05E018069908F083
:1033500057FA0323EA1C9A4300D16BE7034B049905
:10336000E01808F0D5F865E70424ECE70400001144
:10337000FFFFFF7FF80F0000F7B505001400402A9B
:1033800021D8002701AE71803780FFF7FEFE0428A8
:1033900016D93A003100FFF7A5FE042810D9368867
:1033A000BC420BD0BD4209D0221CB44200D9321C11
:1033B000064B92B2C118280008F0D2F830B2FEBD18
:1033C000C04300B2FBE703204042F8E704000011CD
:1033D00037B5042204000D0001A81649FFF7CCFF01
:1033E000020004280BD1019BA34208D3AB4204D0B6
:1033F000104901A80195FFF7F9FE01203EBD0E4CD2
:1034000023682000019308F06BFB0199200001392B
:10341000019108F0F5F980235B01E418074B9C4209
:10342000EED10422034901A80195FFF7DFFE002039
:10343000E4E7C0465555000000C007110000081120
:1034400030B589B008F05CF910226946254808F0CB
:10345000CFF8254B009A9A420ED1019B029A0F2B6E
:1034600033D8002101240698013B08D2002900D05E
:103470000292029B013331D10023029325E0551CB7
:10348000F2D102002100EFE710341022200004A93D
:1034900008F0AEF8029B013301D1069B029388230A
:1034A00004995B05C918059B06981A03120B049131
:1034B0000592814203D02B4201D108F0D1F8019B43
:1034C000013B0193019B002BDED1029B002B03D01B
:1034D000049304984168084709B030BDE025014CC9
:1034E0002D03EFE70000011150485936F7B50F4999
:1034F0000F4B0A6804001A4084235B0013430B60DF
:10350000030003271033019300252E00112008F03B
:1035100047FA084B1B683B40AB4002351E43202D49
:10352000F4D1019B40C4A342EED1F7BD5CF0004052
:1035300000FEFEFF64F00040802270B5AD4CAE4B43
:10354000D200002120001C6008F04AF92300AB4A99
:1035500088331A60AA4B1A786E23002A00D01133E0
:10356000E3620A232365A74B1878A74BA0630138B1
:10357000E361C3B2032B01D810232362A34B37228C
:103580006361C823DB00A36123008C331A60082326
:1035900036210F3AE518E16323646264E967043970
:1035A000251DE96725003B26BC352E602500C0356A
:1035B0002B602500C4352A6025000636CC352E60E8
:1035C0002500083EC8352E602500D0352960210031
:1035D000D4310B602100D8310A6021000225E0318E
:1035E0000D6025004221DC35296025001B3EE435B5
:1035F0002E602500E8352B602500EC352A6022007E
:103600000525F43215602200F032116022001831D5
:103610009032116022009432136023003C229833D0
:103620001A60AF23DB002360794B2363032805D89E
:1036300008F0DEF933023537152363609623210045
:10364000FA225B00A360E360C8332361714BFC3155
:103650009200A3640A6062626F4A704DA262732294
:10366000E2656D3A6265A2650232E5644A60022154
:10367000616696218900A166626709210022E166E0
:10368000A2676749674A684E2167E2673560032889
:1036900011D808F0ADF996089EA61023CDE70E23A9
:1036A000CBE70C23C9E720001A259C3005602000D9
:1036B0000735A03005602000A83003602300FA2001
:1036C000F8338000186023006420A43318602300BE
:1036D0005F38AC33186023000338B0331860230020
:1036E000C630B433186023000020B83318602300BC
:1036F0003825FC339D604D4D5A665D644C4D9A648F
:10370000DD619625AD001D624A4D9A675D62F53D0B
:10371000FF3D9D621E25484ADD6618675867D965DA
:103720001966DA67BE23C021444A5B00E250444B6D
:103730004900635004316250C4225200A350FA235E
:10374000E4205B000432A3500432A3503D493E4ABA
:103750003E4BD1603E49800019503E49E938FF3860
:1037600019503D49043019503C491038D1613C4949
:1037700011633C4951633C4911603C49195019009F
:103780003B48F83108603B49D16582213A4A8900BB
:103790005A501A0039490832D1671A003849B432F0
:1037A00011608821374A89005A501A0036498832F8
:1037B0001160364ADA6408F01BF8012008F030F98D
:1037C00070BD200014259C30056020000435A03019
:1037D00070E7200010259C30056020000335A030E4
:1037E00068E720000E259C30056020000235A030DF
:1037F00060E7C0460004FF1FC465FF1FB070FF1FD5
:103800007C45FF1F4A0AFF1F3A07000080C3C90119
:103810009A02000050C300006A180000280A000045
:10382000204E000088130000F009FF1F0040001127
:1038300068100000C4090000DC05000040420F00D1
:1038400010270000FD1BFF1FFC00FF1F0000FF1FD3
:10385000252FFF1F4D32FF1FE530FF1FD91FFF1F10
:10386000F51FFF1FA121FF1F491FFF1FC528FF1FB5
:103870008D2CFF1FD918FF1FD127FF1F3925FF1FD0
:103880004525FF1F491EFF1F011FFF1FC11DFF1FF1
:10389000F7B50B0CFF270122009300233C001E000C
:1038A0001D009446019089B262469A40100008407B
:1038B00018413618B6B2FF2F02D1012E00D19FB2A7
:1038C000009802401A41AD18ADB2FF2C02D1012D73
:1038D00000D19CB20133102BE6D10320012E07D179
:1038E000012D04D1019B2401E4191C700138FEBD97
:1038F000102EFCD10238102DF9D00230F7E710B5A8
:10390000064C2378002B07D10548FFF7EFFD05484B
:10391000FFF7ECFD0123237010BDC0468465FF1F37
:103920009865FF1F8865FF1FF0B58BB00D00012360
:103930000190102936D8FFF7E2FF00231A001B4838
:10394000C15C01335218102BFAD1023B002A29D056
:10395000174B184C1F68002306A9E25C1600FA5C9E
:1039600056405E540133102BF7D102AA07F080FDB8
:103970002A0002A9019807F073FE07F079FE236878
:103980001B18236007F074FE63681B18636007F060
:103990006FFEA3681B18A36007F06AFEE3681B189C
:1039A000E360002318000BB0F0BDC0469865FF1F10
:1039B0001C44FF1F8865FF1F0223F0B50124574EEA
:1039C000574D3370574B2C701B688FB0552B10D050
:1039D000082006F001FB00280BD0002321000093F3
:1039E0000420514A07F09CFF8023DB059C62FFF70F
:1039F00027FD002006F088FD08F01AF8FFF79CFD6F
:103A000007F0DEFE1F2201240021484B0EAF1A7082
:103A1000474B1C70474B1970474B19689143163A36
:103A20000A431A60602219689143403A0A431A60B7
:103A300008F026F807F054FFC120FF213F4B80001B
:103A40001A588A431A50C522920098588843BF39A1
:103A50000143995098583A4908408021C9010143CF
:103A6000802099509958C0050902090A01439950CC
:103A700080213448490107F09BFF0323220032498B
:103A800001940093314807F043FF2C22304903A8EA
:103A900007F066FD03AC61782078023406F0C2FAC4
:103AA000BC42F8D10121002006F0D6FB294B2A4A5E
:103AB000196803201140A022D2020A431A60802212
:103AC000196892040A431A601968244A1140802236
:103AD00092030A431A60224B224A934200D80120E3
:103AE00007F00EFF07F0E4FF07F0FAFC307807F06C
:103AF000B7FE2878C0B207F04BFD07F0A9FE0A49CF
:103B0000042007F0A5FC06F0CBFC00F09FF800F0C5
:103B10003FFE00F00BFA00200FB0F0BD4A0AFF1F75
:103B20007C45FF1F34F000403B000108480AFF1F9E
:103B3000490AFF1F680AFF1FBCF0004000E100E0D7
:103B4000FF00FFFF8045FF1F0458FF1F8055FF1F28
:103B5000F0BA001114F00040FF7FF8FFFFFF9FFF55
:103B6000B070FF1F0080FF1F70B500252849294A4B
:103B700029484D6308CA1B051B0DED188242F9D177
:103B80000022264B8B63264B08211A628022254B8C
:103B90009205DA67244BDA688A43DA60234A12789E
:103BA000012A03D09A6822490A409A600121EE2432
:103BB0002048E40002686C438A430260DA681120FE
:103BC0008A43DA6007F064FF112007F0C1FC11207E
:103BD00007F05EFD184A200C0400642390420AD8C6
:103BE000FA220023D200904205D9144B0A21C018B2
:103BF00007F016FDC3B2124A1372124BD4801B7821
:103C0000002B04D1104B1021187807F051FC70BD27
:103C1000000005408805054000060540FF01000042
:103C200000F0004004E100E03CF000404A0AFF1FC1
:103C3000FFDFFFFF00380040B70B000030F8FFFF48
:103C40000063FF1F3865FF1F2863FF1F002210B5A8
:103C50001100112007F0DCFC10BD0000F8B50023B6
:103C600001250826394F3A4C3B62E3681120AB43EB
:103C7000E360E368B343E36007F06AFC112007F0F8
:103C800007FF112007F0A4FD4023226829001343F9
:103C9000236080236268DB02134380226360A36891
:103CA00007201343A360A3682A4A1340A36080231C
:103CB000A2689B0113431022A360236C93432364E7
:103CC000236C2B43236480235B003B62226B224BDB
:103CD0001A402263626B1A406263A26B1A40A263AD
:103CE000E26B1340E3631D4AE3681340E36006F0B0
:103CF00083FA2900072006F0AFFA8021184A112024
:103D0000536C0B43536407F05BFEFD21154B164AC1
:103D100089005A508023C720626B5B03134363639F
:103D2000E36880003343E360E368104A1D43104BAF
:103D3000E56019581140802212020A431A5080226D
:103D400092051A600B4B5E63F8BDC04600F0004060
:103D50003CF00040FFFFDFFFEFFFEFFFFFFF7FFFC3
:103D6000003800400000FF1F693B0011FF00FFFF0B
:103D700000E100E00000054030B503A804880B20F6
:103D8000002C0ED14968074D087849780902014393
:103D90000A20A94205D1012120001980024B1B7A7B
:103DA000137030BD192A00000063FF1FF7B515001E
:103DB00008AA16884A680F4F1478527812022243D4
:103DC0000A24BA4214D10122DBB2019200962A00E1
:103DD00007F0B6FA041E0BD1074B1B68002B07D067
:103DE00068782A78000210434242504101309847D7
:103DF0002000FEBD022900008462FF1F30B50125AE
:103E000003790400BFB02B4212D00A49408806F063
:103E100003FE28420CD06A46074B69465B8D5580ED
:103E20001380064B60881B7A1371002203F0BAFEE0
:103E30003FB030BD7C62FF1FC041FF1F0063FF1F0A
:103E400010B50549054806F09DFD0421044A0548C2
:103E500006F05AFD10BDC0467C62FF1FFFFF000048
:103E60001CBB0011C041FF1F10B5024804F01CFD2F
:103E700010BDC046FD3D0011062310B58370103300
:103E80000371443B43712A3383714433C37100236C
:103E90000222012103720E4B027041701C88817254
:103EA0004472197A0273C1729A784273DA78827313
:103EB0000322C2731A7902745A7942740C228274F2
:103EC0009A79C274DB7903751123C370152010BD74
:103ED0000063FF1F10B5142007F0EAFB124B1422F9
:103EE0000021186007F0CCFC002007F059FC0120ED
:103EF00007F0FEFC022007F083FD032003F078FFAB
:103F0000042005F08DFF052003F0B6F9062003F02C
:103F100083FE072001F0DEF8082006F0D5FC09201A
:103F200000F0B6FE10BDC0468862FF1F10B507F056
:103F300097FD012007F0DCFA07F03AFC002010BDE5
:103F4000094B10B50400984205D0012904D1200086
:103F5000064906F017FD10BD0229FCD1013904F015
:103F600061FC0028F3D0F6E7FEFF0000AE62FF1F01
:103F700070B50D7A100004AA2C0016881022144087
:103F8000154220D1002E20D10A78022A18D14A6881
:103F9000517815780E4A09022943914205D00D4AFD
:103FA000914209D01C800A2404E014220A491A8094
:103FB00007F056FB200070BD0C2208491A80F7E775
:103FC0001C800124F6E70824F4E70B24F2E7C0463E
:103FD000F3FF0000F4FF00000044FF1FF8BB0011D6
:103FE00010B504000749084806F0CCFC074804F067
:103FF0009BFB0020E40704D50721054A054806F08D
:1040000083FC10BDAE62FF1FFFFF0000413F0011A7
:1040100060BB00110442FF1F00B50C4BBFB01A7803
:104020000B4901A800F0E8FB6B4680B258800028DD
:1040300009D06A46074B69461B881380064B00224D
:10404000188803F0AFFD3FB000BDC0468C62FF1F73
:104050008D62FF1F5E42FF1F5E43FF1F00B50C4BCA
:10406000BFB01A780B4901A801F0DEFC6B4680B2A4
:104070005880002809D06A46074B69465B8D13803B
:10408000064B0022188803F08DFD3FB000BDC046EE
:10409000B662FF1FB762FF1F0442FF1F5E43FF1F90
:1040A000F7B50E00377A1C0008AB11003D001A88E6
:1040B00020231D401F423CD13378022B3BD1736833
:1040C0001F785B781B023B431E4FBB4208D01E4F3C
:1040D000BB4214D01D4DAB4221D00A252800FEBDA5
:1040E000002A2AD1142C2AD82200F06807F0B8FA46
:1040F000174B1C70012CF1D9FFF7B0FFEEE7002A37
:104100001BD1202C1BD82200F06807F0A9FA114B14
:1041100004211C70104B187807F0CAF9DEE7E3B2EF
:104120000124009201940A00310007F009F905000A
:10413000D4E70825D2E70125D0E70B25CEE70D25EA
:10414000CCE7C046F3FF0000F4FF000002290000A6
:10415000B662FF1F8C62FF1F2863FF1F07B5074B66
:1041600001A9188803F00AFD172805D1044B1E2267
:104170004021187807F094FA07BDC0465E43FF1F40
:104180002863FF1F70B5160004AA148805AA1578C5
:104190004A685078117800022A4A08438018052896
:1041A0004BD807F025FC03131E29343F0720032CAE
:1041B0000BD80422121BAA4200D92A0022491A80D5
:1041C0003000091907F04CFA002070BD0720112CAF
:1041D000FBD81222121BAA4200D92A001B491A80BE
:1041E000EEE707200E2CF0D80F22121BAA4200D9AE
:1041F0002A0017491A80E3E70720032CE5D8042298
:10420000121BAA4200D92A0012491A80D8E70720B7
:10421000032CDAD80422121BAA4200D92A000E4924
:104220001A80CDE70720032CCFD80422121BAA4204
:1042300000D92A0009491A80C2E700220A201A8000
:10424000C3E7C046DCD5FFFFABBB0011D462FF1F44
:104250009BBB001196BB001191BB00118CBB0011E0
:1042600010B50D21024A034806F04EFB10BDC046B2
:1042700080BB00117442FF1F37B5012000F0CAF85F
:10428000204D214BEA89287C9A422AD1042201A997
:1042900000F074F9040000F031F9002C30D16B46C5
:1042A00099882B68C9BA4B432989184A1B145B1893
:1042B00053806B46D9886B6849BA89B24B43698988
:1042C0001B0C5B181248191C1BB2834200DD011C39
:1042D0000B0400D500211388918001331380200046
:1042E0003EBD0223002101AA00F01AF96A4604002B
:1042F00002230121287C063200F012F90443CAE7A8
:104300000124ECE7E862FF1F830500000063FF1F44
:104310000F27000037B5012000F07CF81E4D072262
:104320006946287C00F02AF9041E31D16B461B78BF
:104330007F2B2DD800F0E2F86B46D878F0230204EA
:104340001B031A406B469B8814495BBA9BB21A4305
:104350002B68000953432A891B0C9B184B806B4622
:104360005A789B7812031B011A436B68024353432C
:104370006A891B0C9B181AB21B0402D58C80200082
:104380003EBD074B9A4201DC8A80F8E78B80F6E756
:1043900000F0B4F80124F2E7E862FF1F0063FF1F9A
:1043A0000F27000010B50F4C237C002B0CD0382BAE
:1043B0000BD1012000F02EF8CC22AC21207C920100
:1043C00000F028F900F09AF810BD074BE2899A42F4
:1043D000FAD1012000F01EF80021207C00F0FAF84C
:1043E000F0E7C046E862FF1F8305000010B5084BE8
:1043F0001A7C002A09D05B69002B06D09847041E5E
:1044000001D0FEF7FDFD200010BD0124F9E7C046F4
:10441000E862FF1F70B500210600162005F058FF66
:104420000121152005F054FF07F03AFA0400092095
:1044300007F0CEF900222B4B2B4DDA6661321A6061
:1044400019685B3A9143002E28D0023A0A431A6059
:10445000AC4209D10A22DA6107321A6200221A63D9
:104460009A630132DA6370BD204A944203D11E225E
:10447000DA610532F1E71E4A944203D13022DA6153
:104480000632EAE71B4A944203D14322DA6108323A
:10449000E3E7194A9442E1D16922F7E702220A438D
:1044A0001A604622AC4203D0104A944204D19422AE
:1044B0005A6106329A61D1E70D4A944201D1E6224F
:1044C000F6E70C4A944204D13422FF325A610D328D
:1044D000F0E7094A9442C1D1E62252005A610A32F9
:1044E000E8E7C046005000400024F4000048E8011E
:1044F000006CDC020090D00300D8B80510B5002491
:10450000064B0920DC6607F023F82100162005F091
:1045100073FE2100152005F06FFE10BD0050004015
:10452000F8B51C000023134D0F00EB666860160001
:1045300007F0E6F801238022EB6623002F6152008A
:10454000013B08D207F064FA08200B4A1168002CDE
:1045500003D12000F8BD2A61F2E72B6F034203D09C
:104560002B69013C3370013613685B1A012BEED9BD
:104570000124EEE7005000406008FF1F002370B5E3
:10458000124D1400EB6668600E0007F0B9F80123C5
:104590008022EB6623005200013B08D207F038FA74
:1045A00008200B4A1168002C03D1200070BD2A613D
:1045B000F2E72B6F034203D02B69013C33700136C5
:1045C00013685B1A012BEED90124EEE7005000407E
:1045D0006008FF1F002370B50C4C0D00E36660609F
:1045E00007F08EF80123E366256107F011FA8020B9
:1045F000074A80001168636B034205D113685B1A98
:10460000012BF8D9012070BD0020FCE700500040CC
:104610006008FF1F002370B5134C0E00E366606056
:10462000150007F06DF80123E36626610F33626B16
:104630001A42FCD02B0A23611023626B1A42FCD071
:10464000EDB2256107F0E4F98020084A8000116886
:10465000636B034205D113685B1A012BF8D9012063
:1046600070BD0020FCE7C046005000406008FF1FFE
:10467000002370B5124D0C00EB666860160007F061
:104680003FF80123A619EB660F33B4420ED107F0B1
:10469000BFF980200B4A800011686B6B03420CD17C
:1046A00013685B1A012BF8D9012070BD22782A61AA
:1046B0006A6B1A42FCD00134E7E70020F5E7C046F8
:1046C000005000406008FF1F0A4B0B4A19689068B1
:1046D000884202D980235B04C918536891601B1A71
:1046E0005B181168D80B5B0440185B0C10605360BA
:1046F0007047C04628F000401863FF1F10B51B4BE1
:104700001A793F2A01D93F221A711979184A194892
:10471000117018221849028018480A8002804A80C5
:104720009A791748802402800C208A800132424303
:104730002401101CA24200D9201C124AC8801080FB
:104740005A79002A01D101325A711A7A012A01D804
:1047500002221A725A791B7A0B4853430A21584392
:1047600006F05EFF094C206010BDC0460C63FF1FC1
:10477000480AFF1F5C43FF1F2845FF1F5A43FF1FC6
:104780000465FF1F5843FF1F710200002C63FF1FC9
:1047900010B507210020FEF71BFE124C002807D1A0
:1047A0000C222000104906F05BFFFFF7A7FF10BDA9
:1047B0000C2220000D49FEF7DFFD0C2804D00C224E
:1047C0002000094906F04CFF094C0C222000094941
:1047D000FEF7D2FD0C28E8D00C220021200007F0C3
:1047E0004FF8E2E70C63FF1FECBB0011FC0C00006C
:1047F000E862FF1FF50C0000F0B504000E00150084
:1048000085B0002A00D1BBE00878002120706170DB
:10481000262800D184E00FD8072805D807F0E8F84B
:104820005A3535353588968F232800D1BFE02528A5
:104830005ED0FF23637098E0712800D18DE01ED810
:10484000562851D0602800D19CE05528F1D1013A7A
:10485000874D0C2A46D8002A0AD0711C280006F081
:10486000FFFEFFF74BFF0C2228008249FEF7BEFC3B
:104870000C222900601C06F0F3FE0D2030E07228A7
:1048800000D174E0DC2800D1A9E0DB2800D0C3E02F
:10489000042DCED9B278737812021A43F378102718
:1048A0001B041343327912061A430192052D05D0D9
:1048B0006F1F3A000198711D06F0D2FE05223100EB
:1048C000200006F0CDFE3A000199601D06F0C8FEFA
:1048D000781D05E00C222000674906F0C1FE0C207F
:1048E00005B0F0BD0C22B8E70C226449604DB5E775
:1048F000013A634D0C2A11D8002A08D0711C2800F7
:1049000006F0AEFE0C2228005E49FEF76FFC132273
:104910002900601C06F0A4FE1420E1E70C22EDE75C
:10492000574D1322280006F0ABFFFEF769FBEEE7B8
:1049300005225549601C06F093FE0620D0E712229E
:104940005249601C06F08CFE1320C9E7082250492A
:10495000601C06F085FE0920C2E77178F72900D9AE
:1049600067E74C4B188801F0BFFC0220B8E700F065
:104970009DFB012D02D07278474B1A6006F060FE55
:104980000020ADE7013A454D062A0ED8002A05D091
:10499000711C280006F064FE00F0C0FF062229000A
:1049A000601C06F05DFE07209AE70622F0E7013A58
:1049B0003B4D042A11D8002A06D02800711C06F0AD
:1049C000CFFD384B1B68AB60FFF77EFE0422290049
:1049D000601C06F045FE052082E70422EDE7022A6E
:1049E00000D826E773786370B378A37077781B02DA
:1049F0001F43032A05D0033D3900AAB2F01CFEF77D
:104A0000F5FB10223900E01CFEF7B6FC0300033072
:104A1000002B00DB64E70DE7DA2800D009E7042D5E
:104A200000D806E7B37872781B021343F2781204B9
:104A30001A4333791B061343082D16D9B2797179BD
:104A400012020A43F17909041143327A12060A4329
:104A500003921A601B68052231002000039306F0C0
:104A6000FFFD0422601D03A973E7FE226270F1E7D7
:104A70000C63FF1FFC0C0000F8BB0011ECBB001125
:104A8000E862FF1FF50C0000F462FF1FD462FF1FF5
:104A90009C44FF1F5E43FF1F34F00040F943FF1F9B
:104AA0001863FF1F28F0004070477047013870B549
:104AB000042809D806F09CFF0309250812001B4BA7
:104AC0000221187806F0F4FC70BD184B0821187804
:104AD00006F0CEFF0022164B1A72F5E70024144BA5
:104AE000124D08211A6828781C8106F031FE210039
:104AF000287806F04DFF012000F04AFE00F00EFF7E
:104B0000E2E70A4B0821187806F0B2FF0948FFF7E0
:104B1000B3F9094B094A9B7900209380084A138016
:104B20008022034B52001A81E6E7C0462863FF1F2C
:104B30002C63FF1F6743FF1F0C63FF1F2845FF1FE8
:104B40000465FF1F020010B5094B0A32094C92B2EE
:104B5000DA815A8298811882207802F02BFA042296
:104B6000054B012120781A7006F0A2FC10BDC0464A
:104B70002644FF1F6665FF1F6565FF1F10B50129ED
:104B800009D1054B1B78002B05D02622034B044886
:104B90005A72FFF7D7FF10BD3865FF1F2C63FF1F48
:104BA000C409000010B5164C0A210223E05E06F08D
:104BB00037FD00B200F008FE0423E05E642106F039
:104BC0002FFD012100B200F06FFE237A0024132292
:104BD00020009A426041C0B200F0E8FD032000F0DE
:104BE000ADFD200000F0BEFD064B187805384342AD
:104BF0005841C0B200F0CCFD00F090FE10BDC046A0
:104C00000063FF1F6565FF1F0300F0B50A4D8E1896
:104C1000B14202D152008018F0BD0C782F682409EF
:104C20003C5D0F271C700C7801313C402F683C5DC7
:104C30005C700233ECE7C0465443FF1F10B5114BC4
:104C40001A781870002A0ED000280BD10E4B1A7853
:104C5000062A07D85423D340DB0703D50B4B18781B
:104C600002F0A8F910BD0028FCD0074B1B78012BDF
:104C700002D0033B022BF5D8044B0121187806F033
:104C800017FCEFE73865FF1F6565FF1F6665FF1FAF
:104C9000F7B5614D614A62492870082005F0DEFBD6
:104CA0000121022005F0D8FA022005F0C1FB012104
:104CB000002005F0D1FA002005F0BAFB00F058FE04
:104CC000FEF79EF906F04CFE032256495648FFF7C0
:104CD0009BFF2D24030004221C7054490130FFF770
:104CE00093FF30230222047043708370504C514B69
:104CF0002000DA8706F01CFE022815D006222000CC
:104D00004D49FEF739FB06280ED00321200006F09E
:104D1000DFFD8D23E3706E3B2371062219332000E3
:104D200045496371FEF762FA0D23444F444C454EEA
:104D30003B70013B0422300043492370033B637006
:104D4000019606F08DFC2D23012240494048A371B5
:104D5000FFF75AFF01223F49FFF756FF012234496E
:104D6000FFF752FF0020FFF769FF3B4E3B4A01214E
:104D70003B4B1278307802F0DFF8230000213A78BC
:104D8000307802F0D9F801222178364B01391A70B7
:104D90000020019AC9B205F0D5FC334B1A68552A98
:104DA00030D100221A60314B3C3231485A72FFF741
:104DB000C9FE2021287806F0ABFC0120404205F016
:104DC0000DFD0120404205F0A9FDFFF749FAFFF76C
:104DD00037F800F091FC01204042FFF701F9012073
:104DE00006F056FDF72001F063FA0121287806F05D
:104DF0005FFB287802F03AFA1E4806F019FCFEF72D
:104E00002DFFF7BDFA210B4B1B4A49019981DA812D
:104E100019825A82CDE7C0462863FF1FA94A0011B4
:104E20007D4B00119C44FF1FD462FF1FF462FF1FE3
:104E30006509FF1F2644FF1FADAC00003465FF1F4E
:104E40001565FF1F1765FF1FABBB00116709FF1F2B
:104E50001C65FF1F6609FF1F6665FF1F8643FF1F56
:104E60006743FF1F0665FF1F34F000402C63FF1FE0
:104E7000C40900003863FF1F4A1F0000F8B50A008C
:104E800020230D001A4019423AD0484B1B78002BC2
:104E900023D0FFF719FC464C464E6368727AC31A5A
:104EA000934202D36060FEF7D9FE327A217A531E14
:104EB000DBB2994214D1FFF775FA637A002B09D05F
:104EC000013BDBB26372002B04D170796433584329
:104ED000FFF738FE237A0133237220206840F8BDA3
:104EE0009142EAD300232372FFF780FAFFF75AFEBC
:104EF000314F3800FEF7C0FF390006F081FBDCE7D8
:104F00000BB2002B0ADA2D4B187806F031FD002881
:104F100001D006F0DDFD80200002DFE702242142FF
:104F200006D0234B01201A72FFF788FE2000D5E738
:104F30000B0715D5FFF7C8FB1D4A1E495368497A70
:104F4000C31A8B4202D35060FEF788FEFFF74EFA79
:104F5000FFF728FAFFF726FE00F0E8FB0820BDE780
:104F60001024214206D0114B1B78002BDED1FEF716
:104F70007BFFDBE7012421420AD0114800F06EF8E4
:104F800006F096FC072000F01FFC00F0C7FCCDE700
:104F90004024214202D0FFF7E1F8C7E704240800CB
:104FA000204021429BD0FFF737F8BFE73865FF1F4D
:104FB0002C63FF1F0C63FF1F6743FF1F2863FF1F46
:104FC0004C43FF1FF0B51B4B1B4F1B883A88040056
:104FD0001A4E1B4D85B09A420DD832889A420AD398
:104FE000184B1A882B889A4205D1174A174B1288FA
:104FF0001B889A421BD0052001F0B0F93B8802AA19
:1050000013803388019053802B88114D93800F4B70
:1050100002A91B88D3800F4B2A78188802F0CCFE97
:105020000D4B08212878019A1C7006F039FB05B059
:10503000F0BDC0460265FF1F5C43FF1F5A43FF1FC0
:105040000465FF1F0065FF1FFE64FF1F5843FF1F1D
:105050006665FF1F5E43FF1FFC64FF1F13B50C4B0B
:105060001C78002C11D1002801D00A4B18600A4A84
:105070000A4B11780A4A10780A4A01920A4A0092A9
:10508000002205F057FA200016BD1124FBE7C046A8
:105090006565FF1FF864FF1F6465FF1F5465FF1FF0
:1050A0006665FF1F4065FF1F4465FF1F10B5064B77
:1050B00012201B78052B06D1044B13221988044BB0
:1050C000187801F027FB10BD6565FF1F5E43FF1FC9
:1050D0006665FF1F10B500240122114B5242187063
:1050E000104B1C70104B1A8002F0C0F804220F4BBA
:1050F00021001A700E480C3206F0C2FB102221006B
:105100000C4806F0BDFB07220B4B1C600B4B1C70C0
:105110000B4B1C700B4B1A700B4B1C7010BDC04618
:105120006665FF1F6565FF1F5E43FF1F6465FF1F08
:105130005465FF1F4465FF1F4065FF1F1465FF1F77
:105140001365FF1F6043FF1F1265FF1FF8B5174C63
:105150000600257806A814240078052D23D1B41F55
:10516000134FA5B21824BD421DD88D1FADB2BD424C
:1051700019D8FA256D00AA4215D21D000D4F0A3D1F
:10518000ADB2BD420FD80C4C26800C4C21800C498E
:1051900000240A800B4A1380FFF714FF0A4B0421F6
:1051A000187806F065FC2000F8BDC0466565FF1F55
:1051B000790C0000750C00005C43FF1F5A43FF1F71
:1051C0000465FF1F5843FF1F6665FF1FF0B50BB254
:1051D0000D0089B0002B00DB76E1A64E307806F09A
:1051E000C7FB041E55D00378A22B00D127E1D02B9A
:1051F0001AD0912B4AD143780E2B47D19E4B8288EF
:105200009A4243D19D4A83681278052A3ED10320F1
:1052100018567F283AD09A4B1B68002B36D05B6813
:10522000002B33D0984731E0807807282ED806F03D
:10523000DFFB042D1D444479ADDD6378002B11D1D3
:105240000622E11C8F4806F00BFA01218B4B1970E6
:105250008D4B1A78002A5BD08C4B307801F06CFEB5
:10526000002855D00722854B1A7051E0617800293B
:10527000F8D1E378002B11D0854A864B127830782C
:1052800001F05AFE60706378002BEBD1200006F02D
:105290001FFC80200002684009B0F0BD774B1B78EE
:1052A000022BF3D00121307806F012FA0028EAD15F
:1052B0000121307806F0FCF8E5E76378002BD1D1C6
:1052C0006E4F032807D13B78052B02D101333B7089
:1052D0001EE00223FBE7704B1A88704B0293002AF2
:1052E0000BD01B78002B03D00121307806F0D8F9C1
:1052F0003B78062B04D1013BE9E7029B1A70F7E7E4
:10530000042B41D10121029B3078197006F0D0F8AE
:105310005B4B1B68002BB9D01B68002BB6D0574ADB
:1053200010787FE76378554F002B27D10622211D87
:105330005B4806F095F962895A4B5B491A80A2894D
:105340005A4B1A80E3890B800521397058490A802D
:10535000584A1380228A584B1A80584B1B78012BCD
:1053600009D11F2000F0FAFFFA22920042430421E3
:10537000307806F095F90022484B75E7312B00D0C4
:1053800070E70022454B1A700323A0E70622002194
:10539000434806F075FA0023454A04211380454A24
:1053A00030781380444A138006F062FB082130787D
:1053B00006F05EFBA379083B5A4253412F4A033360
:1053C0001370314B1B78002B06D0344B30781A7891
:1053D000002A06D001F0EEFD0122324B52421A8023
:1053E00096E70121197006F063F8F5E70821307897
:1053F00006F03EFB6378002B00D047E72C4B2E4F86
:105400000293E388029A042113802A4B3078039395
:105410002389039A138063893B8006F059F9002899
:1054200000D033E7264B1B68002B00D12EE70399F1
:1054300002983A88098800881B68984726E74379CC
:10544000132B00D022E70389012B0AD11D4B1B78B7
:10545000022B06D10821307806F00AFBFFF726FE62
:1054600014E7052000F07AFF08210200307806F0EA
:1054700017F90BE76665FF1F051400006565FF1F40
:10548000F864FF1F3965FF1F8643FF1F6743FF1F37
:105490003465FF1F1565FF1F3665FF1F3865FF1F49
:1054A0000765FF1F5E43FF1F0E65FF1F1065FF1F8F
:1054B0000265FF1F0065FF1FFE64FF1F0665FF1FDB
:1054C000F464FF1FFC64FF1F8020C001014200D074
:1054D000E1E6CB0731D5324B1B78002B1DD0314E86
:1054E00005AC3378052B1AD1023B23702E4B2100DB
:1054F0001B7823722D4B1B7863722D4B187801F0AB
:10550000BFFC002809D007202A4B30701B68002BF5
:1055100003D01B68002B00D098470120BBE60E206B
:10552000254B06221B7825492370254B1B78637079
:1055300002ABC01806F094F8D8E702230800184020
:10554000194209D0174B1B78052B03D11D4B188826
:1055500005F0F6FF02209EE60424214203D0FFF767
:1055600031FD200097E6082308001840194200D1B9
:1055700092E6154B1C78012C03D0022C0DD008208C
:1055800089E6124B124A134913481B88128809886E
:1055900000880094FFF7DAFDF1E7FFF787FDEEE7FB
:1055A0003865FF1F6565FF1F6043FF1F1265FF1F02
:1055B0006665FF1FF864FF1F1465FF1F6143FF1F2F
:1055C0001365FF1F5E43FF1FFC64FF1F5843FF1F4F
:1055D0000465FF1F5A43FF1F5C43FF1F10B502A85D
:1055E00004880B20002C10D14968087849780902FA
:1055F00001430C48814209D1022119800A4B598884
:105600001170DB7800205BB2537010BD074C0A208C
:10561000A142FAD102211980034B998811705B795C
:10562000F0E7C0466E2A00000063FF1F6F2A0000EB
:10563000F7B5150008AA16884A680F4F14785278F3
:10564000120222430A24BA4214D10122DBB201928F
:1056500000962A0005F074FE041E0BD1074B1B6850
:10566000002B07D068782A7800021043424250414C
:10567000013098472000FEBD022900007865FF1F19
:1056800030B5012503790400BFB02B4227D015495E
:10569000408805F0C1F928420DD06A46124B694690
:1056A0005B8D138002235380104B5B88938060884E
:1056B000002202F077FA0E49608805F0ADF9C007C4
:1056C0000DD56A460B4B69461B8813800223538015
:1056D000064B9B8893806088002202F063FA3FB0FB
:1056E00030BDC0467065FF1F8843FF1F0063FF1F6A
:1056F0006865FF1FE243FF1F10B5074C07492000F4
:1057000005F040F92000064905F03CF90721054A5B
:10571000054805F0F9F810BDFFFF00007065FF1F98
:105720006865FF1F78BC00118843FF1F10B5024851
:1057300003F0BAF810BDC0468156001170B55F2560
:10574000082607498400CA788B7840012A40B34371
:105750003440A843234302438B70CA7070BDC046D7
:10576000F943FF1F010043B204205A0002409B008E
:105770000C3003401A43152310B5044CE0789843CD
:10578000143B0B4018430243E27010BDF943FF1F66
:1057900010B5054B082419790A00A243002801D04E
:1057A00022000A431A7110BDF943FF1F10B5054BC3
:1057B0004024D9780A00A243002801D022000A43DD
:1057C000DA7010BDF943FF1F082170B5314D040098
:1057D000AB780B40AB70304B984204DD67232B70E5
:1057E000473B6B7070BD2D4B984203DAE0232B7062
:1057F0003A3BF6E700232B706B7083B21A002848FF
:105800005F3292B2274E82422CD9002C03DA5B42DF
:105810001CB204232B70053420B20A2105F000FFCE
:1058200004B2FA239B009C4231DB08232A781343FD
:105830002B706421200005F0F3FE0A2100B205F070
:105840009FFF09B22A78735C13432B700A21200052
:1058500005F0E6FE0A2100B205F092FF09B2735C82
:105860006A780AE06970002CDBDA5B421CB2042320
:105870002B70F3226B78092CE8DC13436B700A2140
:10588000200005F07DFF09B2735CAB70AAE7632CC2
:10589000CFDCEEE7F943FF1F1B4E00001DFCFFFFAE
:1058A0002A0800009FBC00110823F7B5194FCD004E
:1058B0003E7904001E403E71EDB2632806DD5F3381
:1058C00033433B7120231D437D71F7BD0300093332
:1058D00005DA20235B4233433B71A623F3E70E4BEB
:1058E000019300280BDA0423444224B23B710A21BD
:1058F000200005F045FF019B09B25B5CE3E7092846
:10590000F5DD0A2105F08CFE019B00B21B5C1E43F5
:105910003E71ECE7F943FF1F9FBC001170B5104BBF
:105920001B78002B1AD00F4E0F4D06223100280095
:1059300006F0C6F8002811D0062231000B4C2800D2
:1059400005F00EFE0020FEF765FD072221003E2037
:10595000FEF78EFE002801D0FEF7D0FD70BDC046D8
:105960008365FF1FF943FF1F7D65FF1F7C65FF1FD8
:10597000002010B5FEF74EFD0D223E200549FEF732
:1059800077FE0023984200D13E33034A1370FEF79E
:10599000B5FD10BD92BC00118365FF1F0200F0B57C
:1059A00001270A480A4E51188B1A002B00DCF0BD63
:1059B000082415784308684038404000805B013C6B
:1059C00058406D08002CF5D10132EDE7FFFF0000D3
:1059D000B0BC0011F0B500250F269D4200DBF0BDE4
:1059E0004C5D070944403440A400A058013578407C
:1059F000F3E70000F0B589B06A460D000B000F27F1
:105A0000110010351C780133260024093E40167021
:105A100054700232AB42F5D12023024AFFF7DAFF7D
:105A200009B0F0BDB4BC0011F0B54E780B7889B068
:105A300036020C00170001901E43012A61D9974BD2
:105A40009E4200D877E001339E421CD1062A17D12E
:105A5000CA788B7812021A430B791B0413434A79D4
:105A600012061A438E4B5A6100221A705A808D4AD0
:105A70005A608D4A9A608D4ADA60002009B0F0BD04
:105A800088225205EEE78A4B9E423CD184498B78AE
:105A9000002B00D0F9E00C2A31D10F22A3789343D8
:105AA000E278120213432279120413436279120638
:105AB00013434B60E279A07912020243207A00047A
:105AC0001043627A12060243CA60E27AA07A120296
:105AD000024378484A81834208D80423704914223B
:105AE00001980B7005F0BCFD1420C7E71201D21815
:105AF00089235B059A42F0D801238B70BDE7022A07
:105B0000FAD00523EAE76C4A01239642E6D1FFF773
:105B1000CDFA052F0CD9E378A2781B021343227922
:105B200012041A4363791B061343644A03931360F8
:105B300005F086FDA1E75A4D2B78002B9DD1AB785F
:105B4000002B00D1A3E02B8901339BB20093B34219
:105B500000D094E0132AD4D9CF7C8B7C3F02122151
:105B600020001F43FFF71AFF874200D091E0002E6C
:105B70003ED1E378A2781B0213432279E96812042C
:105B80001A4363791B06134303930A228B4213D1F2
:105B9000FF23A370E370237163716B89002B0AD11B
:105BA000E37B227C1B0212041343A27B1343039367
:105BB0001B0901336B8100226B89002B8DD0002AD9
:105BC00069D1686837013818000B6B6900030390CE
:105BD000984205D9686105F083FFEB780133EB70DB
:105BE00068681022A11C381805F092FC2E8144E749
:105BF0006F89009A7B1E9BB293423CD1E378A278D6
:105C00001B02134322792E4E12041A4363796C68E7
:105C10001B0613433100042204A8039305F020FD62
:105C2000211D0C2205A805F01BFD012004A94042FE
:105C30001034FFF7DFFE013F012F17D1039A0B232A
:105C40002861824200D049E704223100686805F0EB
:105C50005FFC042203A9686805F0C2FEE968039AA4
:105C6000FF23914200D139E7F73B37E72100FFF7E7
:105C7000C1FE1034DFE70923B742A2D82EE7009B0C
:105C8000B34200D9F9E6072328E7022326E70323D6
:105C900024E7062322E70A2320E7C046FFFE000090
:105CA0000044FF1F00000111FFFF0000504859365B
:105CB00001FF0000FFFF001102FF000034F0004070
:105CC0000C44FF1F10B5034C0B000122210000F013
:105CD0006BFA10BD855E00110B8870B506000D00D3
:105CE0000224162B11D92B000322094900F05CFA7B
:105CF000041E0AD1074B2A881B88191C934200D91D
:105D0000111C300089B200F0EFFA200070BDC046CF
:105D1000B15E0011DE65FF1F10B54A780400013A3C
:105D20000B000220012A07D80A78002A04D0052295
:105D30002000024900F038FA10BDC046DF5E0011B5
:105D40000A7810B50B0004000220002A04D00722B4
:105D50002000024900F028FA10BDC0468B5F0011F8
:105D60000A7810B50B0004000220002A04D0092292
:105D70002000024900F018FA10BDC046F15F001182
:105D800010B5034C0B000B22210000F00DFA10BDE2
:105D90002160001110B5034C0B000D22210000F012
:105DA00003FA10BD9360001110B5034C0B000F22D5
:105DB000210000F0F9F910BDED6000110A7810B56E
:105DC0000B0004000220002A04D011222000024906
:105DD00000F0EAF910BDC046FD600011002310B5C7
:105DE0001322190000F0E0F910BD000010B5034CBB
:105DF0000B001722210000F0D7F910BD4F610011F0
:105E0000002310B51922190000F0CEF910BD0000D2
:105E100010B5034C0B001B22210000F0C5F910BD8A
:105E200089610011F7B584890D0006000121002C5D
:105E300022D000238268D3561778002B1EDA0C2C50
:105E40001AD90C3CA4B2131940880093230002F025
:105E500086FE431E984101307B06DB0F6B703F23AB
:105E6000013C1F40A4B22870AF70AC80002C07D05A
:105E7000B3680133AB6000210800FEBD0020EBE7F2
:105E8000AC60F8E70B7803704B8843704B881B0AB3
:105E900083700B79C370042070470420022B06D155
:105EA0000020537811781B02009A0B43138070472F
:105EB0000B8803700B881B0A437002207047042074
:105EC000009983420AD1537810781B0203430B8058
:105ED000D37890781B02034300204B807047F8B5BD
:105EE0000D004B7801240021461C03702B788B4257
:105EF00001D82000F8BD6B78B01C4F1C012B10D1CD
:105F0000890069184B88022233704B88B9001B0A3C
:105F10007370691805F0A4FB04360434A4B2F9B216
:105F2000E4E7122359436B185A88043132705B88B6
:105F300010221B0A7370691805F092FB1236123496
:105F4000ECE770B5049D14001E00052B01D8042059
:105F500070BD637812781B0213432B80E378A2781C
:105F60001B02134302226B802A71211D681D063E0D
:105F700005F076FBB2B22A81F02AE8D82800A11DEC
:105F80000A3005F06DFB0020E2E7002310B50A7827
:105F90009A4201D8900010BD9A008A1854880133A3
:105FA00004705488DBB2240A447094888470928808
:105FB000120AC2700430EAE710B51100029C062BE9
:105FC00004D004201022142B01D010BD0222227113
:105FD0004B7808781B0203432380CB7888781B0218
:105FE000034363800431601D05F03AFB0020ECE7B9
:105FF00010B50C788B7804315C43E4B20370220056
:10600000013005F02DFB601C10BD0420022B06D1D1
:106010000020537811781B02009A0B4313807047BD
:1060200010B50C000A88023105F01AFB208810BD5B
:1060300070B504000D0004981100012B01D8042054
:1060400070BD167852781202324302800200F83294
:1060500055701470E825002C00D10C35023B9AB223
:106060004280AA42EBD80231043005F0F9FA002050
:10607000E6E70420009983420AD1537810781B0286
:1060800003430B80D37890781B02034300204B809E
:10609000704710B50C000A88023105F0E1FA20883B
:1060A00010BD000070B501211E000420049C0E40AC
:1060B0000B4218D1CB40DDB28D4214D90A49DBB274
:1060C000098899420FD32300F6331D70330058001E
:1060D00011184978165C0902314301332152D9B2B3
:1060E0008D42F4D8002070BD2044FF1F10B50C0075
:1060F0000A88023105F0B4FA208810BD10B50C787A
:106100008B7804315C43E4B203702200013005F067
:10611000A7FA601C10BD10B511000298032B01D81E
:10612000042010BD14785278043B120222430280EE
:10613000CA788C781202224342809AB28280F22A74
:10614000EED80431063005F08BFA0020E9E710B5EF
:106150000C000B8803700B881B0A43704B888370FC
:106160004B881B0AC3708A880430063105F078FA20
:10617000A088043080B210BD0420012B03D1002080
:106180001378009A1370704710B50C000B880370D9
:106190000B881B0A43704A880230043105F060FA0C
:1061A0006088023080B210BDF0B589B003931E4BF9
:1061B000029242000700D05A019102F020F8132504
:1061C000061E2DD0029B01240370019B002B04D0DE
:1061D000001903999847001984B26B461B7A5BB289
:1061E000002B0FDA1021380002F01CFB19250028C3
:1061F00013D130003219E1B202F066FC051E0CD159
:106200000C34A4B2042304AA380005A9938006968E
:10621000948101F0AFFD051E02D0300005F068FA50
:10622000280009B0F0BDC046DC65FF1F70B5050051
:106230000C0000280CD00020814209D01022200040
:10624000044905F00DFA01202B7823736B786373F2
:1062500070BDC046F4BC0011F0B506000D0017007B
:106260001C0085B002291BD00020102907D1022B69
:1062700007D0102B03D115E00020102C08D005B05A
:10628000F0BD69463800FFF7D1FF2A0069460BE0F0
:1062900069463000FFF7CAFF22006946380004E073
:1062A000022BE9D12A003900300005F091FBE6E726
:1062B000031CF72800D9F723032008499AB2013AB2
:1062C0000B80D317034006499B189B100B80D30FFC
:1062D00004499B185B100B807047C0462444FF1F85
:1062E0002244FF1F2044FF1F034B1B888B4202D315
:1062F000024B4000C15270472444FF1FDC65FF1F62
:10630000014B4000185A7047DC65FF1F1722014BF4
:106310001A807047DC65FF1F70B505000E2005F080
:10632000EFF8041E13D0D0230370002306228370DD
:1063300007494570033005F093F9064B2100DA8ACE
:1063400062811B7E2373044B187805F0F9F970BD48
:10635000F865FF1FE865FF1F7444FF1F262803D858
:10636000024B4000C05A70470148FCE72644FF1F1B
:10637000FFFF000070B506000C00094D1C22002133
:10638000280005F07DFA074B1E70074B1C7005F0C6
:1063900007F90123002801D0002312202B7070BDC3
:1063A000E865FF1F7444FF1F0966FF1F70B50500F5
:1063B0000D4C0800E260A16010220021656005F02C
:1063C00007F9012803D11021A06802F058FD10221E
:1063D0000021280005F0FCF8012803D11021606895
:1063E00002F04DFD70BDC046E865FF1F70B5041E8C
:1063F00005D1002903D006220D4805F031F90D4BD7
:106400001D78012D11D1002C05D102221A7005F042
:106410008FF8280070BD00221A70074B1B78FF2BE5
:10642000F7D02000FFF778FFF3E70025F1E7C0463B
:10643000F865FF1FE865FF1F7444FF1F030010B5D8
:10644000002801D1002010BD00780B4A002803D19C
:106450005988D1821B7913761378022BF2D100234D
:10646000984200D103331370044B1B78FF2B01D0EB
:10647000FFF752FF0120E6E7E865FF1F7444FF1FA6
:10648000002911D000280CD04B79012803D14022DB
:106490005242134303E03F221340032802D001205D
:1064A0004B7170474022F4E70800FAE770B5094DD8
:1064B0000100287800280BD0074C0622200005F0A8
:1064C000CFF821002878FFF7DBFF200005F0D8F88F
:1064D00070BDC0460866FF1FE265FF1F00290AD095
:1064E000012808D13F224B799343C02B03D0403B76
:1064F0005A425341981C704770B5174D06002B78CF
:10650000FF2B15D00A2004F0FBFF041E10D0D0236F
:106510000370C83B8370114B11491B784670C370E0
:106520000622043005F09CF82100287805F008F9CF
:106530000C4B1B78012B0DD10B4B1B68002B03D090
:106540009B68002B00D09847084B04211878084A14
:1065500005F0FEF870BDC0467444FF1F0866FF1FBB
:10656000E265FF1F0466FF1F3066FF1F3466FF1FD2
:1065700060EA0000014B98687047C046E865FF1F5D
:10658000014BDB6818687047E865FF1F074B10B5C3
:10659000DA68136801331360054B1878FF2803D0BD
:1065A0008021C90104F084FF10BDC046E865FF1FCB
:1065B0007444FF1FF7B50E0002F0C8F8051E1CD08A
:1065C0000E4B06621F78002F00D10778AB791020A0
:1065D000019304F095FF041E0FD0D0230380C73B26
:1065E0008370019BE91DC3700622043005F038F862
:1065F00021003800E66005F0A3F8F7BD7244FF1FE4
:10660000014B18787047C0460866FF1F054B0028ED
:1066100005D1054B1A78054B002A00D1014B180013
:106620007047C046F865FF1F0866FF1FE265FF1F41
:10663000014B58687047C046E865FF1F024B186859
:10664000431E9841C0B270470C66FF1F421E0300F4
:106650000120152A03D9FF3B5A425341D8B2704753
:10666000F0B51C0000230E0085B0039002920B7061
:10667000029A934201D3002019E0E55C5A1CD2B281
:10668000002DF8D0029851198142F4DC0233DFB2B8
:10669000A35C18000193FFF7D9FF002807D0013D44
:1066A000019A0399EBB233708A4202D1E01905B026
:1066B000F0BDDB19DBB2DBE710B50C0002F09EF891
:1066C00003001220002B03D02100588805F030F879
:1066D00010BD000070B50E4D84006359002B15D01D
:1066E000186A002801D005F02BF92B59586A0028A8
:1066F00001D005F025F92B59986A002801D005F042
:106700001FF9285905F01CF900232B5170BDC04614
:106710001866FF1F1C4B70B504000E00150099424F
:106720000AD11A4B1B68002B01D1122070BD1B68C7
:10673000002BFAD09847F9E7154B994215D1134B26
:106740001B68002B0AD01B68002B07D09847002835
:1067500004D1104B1C70104B1D70E7E7290020007E
:10676000FFF7AAFF0028E1D1F3E7080001F0EEFFF0
:106770000028DAD003780320A342D7D129003000C3
:1067800004F0D6FFD2E7C046FEFF00001466FF1FEC
:10679000FFFF00001166FF1F1066FF1FF7B5040022
:1067A000808801F0D3FF0025A84203D00578A08897
:1067B00002F008F81C4E3378002B1FD0AB421DD1DD
:1067C0001A4B28001978FFF777FF002818D000230C
:1067D0003370A3790820A778A688019304F090FE6F
:1067E000011E0DD0D0230370CA3B8370019B4770FC
:1067F00086808371280004F0A3FF01E0002DE8D11A
:10680000A0880B4B8200D358002B01D0FFF762FF0A
:106810001721A088FFF768FDA08801F027FDA08858
:1068200001F0FEFDF7BDC0461166FF1F1066FF1F99
:106830001866FF1FF0B587B01D000CAB1B88070062
:1068400001930DAB1B88142002930EAB1B8816001E
:1068500003930FAB1B880091049310AB1B88059327
:1068600004F04EFE041E1AD0D0230370CB3B4770B9
:106870008370C670062229000430002D11D004F068
:10688000EFFE019B21006381029B0098A381039B83
:10689000E381049B2382059BA37404F051FF07B09E
:1068A000F0BD04F0EDFFECE7F7B5009308AB1B88F3
:1068B00007000C200D001600019304F021FE041EB9
:1068C00013D0280001F042FF00280FD00078D02319
:1068D0002370C93BA370009B21002381019B67703B
:1068E000A580E680638104F02BFFF7BD014B18788B
:1068F000EDE7C0467444FF1F13B5040064890389A3
:10690000C2888188C0780094FFF7CEFF13BD0000D5
:1069100010B5044C2068002803D005F011F80023BE
:10692000236010BD1C66FF1FA122F0B58188920074
:106930004A43384B384F1B6804009B189D22920035
:106940009B18827989B01A603B68002B5FD01D7854
:10695000324B1B68002B04D05B68002B01D0002059
:106960009847260008363100E079FFF7B7FD237D10
:10697000E0710200E0780493638A29000393238A7C
:106980000293E3890193A38800933300FFF752FF3A
:10699000E378002B0BD1E289A379A18802920196BA
:1069A000E27928000092012201F0DAFEE0703B68F3
:1069B000002B20D0FFF7ACFF194D287800281AD003
:1069C000184B1978FFF778FE002814D02B78E6785A
:1069D00008200793A78804F093FD011E09D0D02357
:1069E0000370CA3B4670837087808671079804F0F5
:1069F000A7FE00232B701721A088FFF775FCA08845
:106A000001F034FCA08801F00BFD09B0F0BD064B8D
:106A10009DE7C0463409FF1F1C66FF1F3066FF1F3D
:106A20001166FF1F1066FF1F7444FF1FF8B50700B3
:106A300008000E0001F08AFE041E18D02620FFF781
:106A40008DFC051E00D12578062004F059FD041E9A
:106A50000DD00021062204F013FFD0232370C23B87
:106A600021006770A370A680E8B204F069FEF8BD4B
:106A7000F0B585B001930AAB1B78070002930BAB0E
:106A80001B7808000D000092039301F05FFE061EC4
:106A900022D0102004F034FD041E1DD0102200214D
:106AA00004F0EEFE2620FFF759FC002800D13078D4
:106AB000D0232370C13BA370009B21002372019B54
:106AC00067706372029BA580A372039BC0B2E372DE
:106AD0000C9BE36004F034FE05B0F0BDF7B50D008B
:106AE000019001F033FE071E20D00E2004F008FDB7
:106AF000041E1BD02620FFF731FC061E00D13E7875
:106B0000D0232380C53B0622A370F91DE01C04F0AE
:106B1000A7FD019B2A0063810123DD401A401D402F
:106B2000210022736573F0B204F00AFEF7BD000085
:106B3000F0B585B0029010000D0017000A9E039377
:106B400001F004FE041E31D0029B002B2ED1039BCA
:106B500002795B0724D5122313430422002E08D1A7
:106B60000B99002905D10C99002902D10D99002912
:106B70001AD01A430D9B2271002B00D0C9E0002EC1
:106B800000D1CFE0002D00D0CCE0606A002801D019
:106B900004F0D6FE1C21300004F00AFD606205E01E
:106BA00002239A430E33D7E793432371654BBA0010
:106BB000D458002C00D1AAE0002E10D0236A002B5C
:106BC00003D11C2004F074FD20625E4BBA00D35840
:106BD000186A002803D01C22310004F041FD0C9BF0
:106BE000002B12D0574CBB001D596B6A002B03D1F0
:106BF000162004F05DFD6862BB00E358586A002867
:106C000003D016220C9904F02BFD0D9B002B11D004
:106C10004C4DBC006659B36A002B03D1142004F01C
:106C200047FDB0622B59986A002803D014220D99B1
:106C300004F016FD380001F089FD051E67D0414BB8
:106C4000BA00D358002B62D01A6A3420002A00D12F
:106C50001C389A6A002A01D0143080B20B9A002A9C
:106C600001D01C3080B25B6A002B01D0163080B29C
:106C700004F046FC041E4AD01822002104F000FE55
:106C80002620FFF76BFB0190002801D12B780193A0
:106C9000D0232370029B200063700A23294EA37027
:106CA000039BBD00A371AB59A780196A1830002956
:106CB00005D01C22A06004F0D3FC200034307359AE
:106CC000996A002907D0030014221433E06002936C
:106CD00004F0C6FC02980B9B002B08D003001C227A
:106CE0001C330B992061029304F0BAFC029873598B
:106CF000596A002903D01622606104F0B1FC6B468A
:106D00002100187904F01CFD3800FFF7E3FC05B002
:106D1000F0BD10220D9B0D991B69A018236204F091
:106D20009FFC2CE70B9B002B00D13FE7012D00D0EF
:106D30003CE7606A002801D004F002FE1C210B9899
:106D40002AE7C0461866FF1F10B5044C20680028CB
:106D500003D004F0F5FD0023236010BD0C66FF1F77
:106D60000B4B07B51A68002A01D100200EBD6946F9
:106D7000531C012012780731FFF772FC0028F4D071
:106D800002780123100018401A42EED0EEE7C04608
:106D90002866FF1FF0B51F4F01203B6887B0002B0E
:106DA00025D09B78059300F0B3FB002821D00A2062
:106DB000FFF7D4FA04000B20FFF7D0FA164B0500BA
:106DC0001E78731E9E413B68F6B2191DD878FFF7F6
:106DD00057FB3B682900DA7A043303929A790193CE
:106DE0000292009033002000059A04F069FB07B07E
:106DF000F0BDFFF7B5FF002805D00620FFF7AEFA7B
:106E000004000720D8E70820FFF7A8FA04000920AB
:106E1000D2E7C0460C66FF1F0866FF1F70B50A4E1A
:106E2000040033780D00FF2B0DD0042004F068FB24
:106E3000011E08D0D0230370CE3B45708370C47010
:106E4000307804F07DFC70BD8444FF1F70B50400F1
:106E500006200D0004F054FB011E0AD0D02303705D
:106E6000CD3B8370054B44701B688580187804F017
:106E700067FC002C01D0FFF767FF70BD0C66FF1F99
:106E8000F8B5264F06003B680D001124002B05D1F4
:106E90000522234B1B78134202D112242000F8BD97
:106EA000204A10241268002AF8D01278002AF5D05F
:106EB000DB0719D52B789A1E012A1AD80C2004F06A
:106EC000F7FB132438600028E8D000230A2243701F
:106ED00029000670023004F0C3FBFFF75BFF041EBD
:106EE0000AD0FFF731FFD9E700F012FB0028E1D10B
:106EF000E4E7002BE2D0D0E70B4B1B78032BCDD17E
:106F00001D20FFF72BFA094B18800028C6D0084B2C
:106F100004211878074A04F01BFCBFE70C66FF1F2A
:106F20000966FF1F2866FF1F0866FF1F0666FF1F12
:106F30003466FF1F60EA0000F7B50193194B140097
:106F40001A78052306000F0012201A4221D00129C9
:106F500020D1154B1D68002D1BD002201F2C18D8E6
:106F6000002C02D0019B002B13D0104B1F221E704F
:106F70006E1C0021300004F083FC019922003000D7
:106F800004F06EFB310020002C70002F06D004F0BE
:106F900047FCFEBD064B12201D68DCE704F0F0FA4A
:106FA000F7E7C0460966FF1F2866FF1F8444FF1FDE
:106FB0002466FF1FF8B50F4E12243368002B17D03C
:106FC0001B780F3C834213D100250B4F02213878E8
:106FD00004F04EFD094B042138781D8004F048FD73
:106FE000074B28001D8033685C7004F0F9FA040038
:106FF0002000F8BD0C66FF1F3466FF1F2066FF1FD0
:107000000666FF1F70B5012823D11B4C2388002B77
:1070100003D01A4A1578002D07D0194B1B68002B96
:1070200002D01878FFF7C6FF70BD3B2B02D93C3B5E
:107030002380F9E7134E0221307804F019FDFA227B
:107040002388920002215A43307804F029FB2580DE
:10705000EAE70B4B1B68002BE6D00B4B1B785B075A
:10706000E2D5084B0221187804F002FD0022024B01
:107070001A80FFF769FED7E72066FF1F0466FF1F2F
:107080000C66FF1F3466FF1F0966FF1FF8B51E4D13
:107090002868002803D004F053FC00232B601B4E0B
:1070A0003068002803D004F04BFC00233360184FF5
:1070B00005243B7818002040234221D0154800F0D9
:1070C0002BFA3B78234213D0202004F0F1FA2860F9
:1070D000002813D02022002104F0D2FB202004F04D
:1070E000E7FA041E306005D02022002104F0C8FB1E
:1070F000002004E0286804F023FC2C601320F8BD75
:1071000000F00AFAF4E7C0462866FF1F2466FF1F56
:107110000966FF1F7844FF1F10B50A4C23681A1E2A
:107120000ED0002808D10130587004F059FA002818
:1071300005D02368002B02D00021FFF787FE012233
:10714000100010BD0C66FF1FF7B5274E0500336811
:107150000191181E21D05C78244F012C30D1FFF70B
:10716000FFFD002825D02000FFF7F8F80400412893
:1071700014D91F4B022118781E4A04F0E9FA1E4B5D
:107180003C3C1C80022233685A703B78002B14D19F
:1071900028000199FFF75AFE0120FEBDFA22920055
:1071A0004243002AEED0124B0221187804F078FAFC
:1071B000E8E7FFF7D3F80200F3E700233B70EBE7C3
:1071C0003B78002BE8D1032004F09AF9011E08D087
:1071D000D0230370CC3B457083703368187804F07B
:1071E000AFFAFFF7B1FDD7E70C66FF1F0466FF1F7C
:1071F0003466FF1F60EA00002066FF1F10B51749C4
:10720000838802008B4220D011D815498B4217D0B9
:10721000144900205B1899B2012907D892681178A7
:107220005A425341D8B2FFF7F9FD012010BD0E4A72
:1072300000209B1807229BB29A424041C0B2F5E75A
:1072400083681878FFF768FFF0E7836899785A78C1
:10725000090218781143FFF777FFE7E70A200000DB
:1072600006200000F8DFFFFFAFDFFFFF014B1870C3
:107270007047C0468544FF1F10B5064C207001F0D2
:1072800041FA207804F0FCF80521207800F062FD36
:1072900010BDC0463466FF1F0BB273B50D00002B46
:1072A00000DBC4E0884B187804F062FB041E0ED0AB
:1072B0000378912B0FD0A22B00D1A1E0834B18783B
:1072C000FF2852D0210004F03BFA00284DD1802045
:1072D0000002684076BD43780F2B76D013D8052B7B
:1072E00070D00E2BEAD18088794B98422BD8794BFD
:1072F00098421BD8784B9842E0D1A3681878591C63
:10730000FFF774F838E03E2BD8D18378032B74D084
:107310006CD8012B6ED0022BD0D1704B1B68002B88
:1073200023D05B68002B20D098471EE06C4BC01820
:107330000C28C3D804F024FB1DC2C2150BC20B0BD2
:107340000B3223C23C00674BC0180728B6D8664BE7
:107350001B68002B09D01B68002B06D02000984723
:107360000AE0A3681878FFF7C7F8200004F0B0FB24
:10737000ADE7A068FFF762F800289FD0F5E7A368A3
:107380001B78002BF1D0554B1B68002BEDD01B68F0
:10739000002BEAD0210055489847EDE74F4B1B687A
:1073A000002BE2D01B68002BDFD021005048F3E710
:1073B000504B1B68002BD8D05B68002BD5D0210028
:1073C0004348E9E7FFF7EAF9CFE780884A4B98425C
:1073D00003D04A4B984200D070E7464B1B68002B05
:1073E000C3D05B68002BC0D02100D5E7153B012B33
:1073F000BBD963E7FFF798FAB7E7FFF77DFAB4E781
:107400003F4B1B78042B07D100236A461380017978
:10741000408800F0C5FCA8E7364B1B68002BA4D0C1
:107420005B68002BA1D00100364898479DE70124F6
:1074300021420AD0294B1B68002B04D05B68002B2B
:1074400001D000209847012043E78B070AD5264B3F
:107450001B68002B04D05B68002B01D020009847EC
:10746000022036E70421280008400D4200D131E710
:10747000254E3388002B21D0013B9BB23380002B5B
:107480001AD1FFF7DBF800280AD0204B1C70164BEE
:107490001B68002B04D05B68002B01D020009847AC
:1074A000FFF7C6F8694601F001FD6846FEF7FEFFEA
:1074B0001D20FEF753FF308004200AE7024B1878A6
:1074C00004F0D6FAF8E7C0463466FF1F8544FF1F74
:1074D0000E20000001200000091000002C66FF1F94
:1074E000FEDFFFFFAFDFFFFF3066FF1F0C20000055
:1074F0000B2000001466FF1F0D2000001320000069
:107500000966FF1FFFFF00000666FF1F0466FF1FDE
:1075100010B501F09BF910BD014B18607047C046D3
:107520003066FF1F0B880020162B01D8172304207C
:10753000014A13807047C046DE65FF1F0020704778
:10754000074A03001188814207D0918800209942A0
:1075500002D101308000101870470020FAE7C046C1
:107560003C66FF1FF0B58F7806000D00C7B01E2FD8
:1075700015D1FFF7E5FF051E03D10024200047B019
:10758000F0BD00223B003100C078009200F0B2FB59
:107590000400A81C00F0D3FBFF23EB70EEE7264BA2
:1075A000062403931B78FF2BE8D0182FE6D87B081E
:1075B000224A013BDB0002929A589446002ADDD011
:1075C000029AD3185B68002BD8D00878002802D123
:1075D0004B78012B02D10624122FCFD107AFAB88F5
:1075E000697800976446AA68A047041EC6D1AB78A4
:1075F000029A5B08013BDB00D318390030005B685E
:107600009847041E0BD1AB78042BB6D0039A3100F7
:1076100010782200009700F06DFB0400AEE76A7856
:10762000002AABD1AA7805A93B88087130000A70FE
:107630004B80FEF747FBA0E78844FF1F04BD001105
:107640001D4B37B5050098420BD000290AD1FFF732
:1076500077FF002805D11948FFF772FF002800D0F6
:10766000058037BD01291AD1FFF76AFF041EF8D043
:1076700001235B420380A378FF2BF2D0FE2B07D0BF
:107680000023E0781422009329001E3300F032FB1F
:10769000A01C00F054FB01235B426380E1E7022958
:1076A000DFD1013901F0BEF80028DAD12800FFF758
:1076B00047FF041EDFD1D4E7FEFF0000FFFF0000FC
:1076C000022210B5074B52421A80074801325A80F5
:1076D0009A80DA8000F07EFA044801F025F8002054
:1076E00010BDC0463C66FF1F657500114176001154
:1076F0000388F7B50400002B02D102252800FEBD47
:1077000042680221137825485268FEF7A5FD00283B
:107710002ED0234F01253A88002AEFD080232188DC
:107720005B0201259B1A9942E8DC0C2003F0C0FFA4
:10773000061E31D03B8822889C4600231800019504
:1077400061469DB2491989B2AA421BD8002801D0CE
:1077500062443A8000233000082208C0210003F070
:107760007FFF104A1368002B13D100251660C5E770
:107770006268022113780C485268FEF76DFD0028FC
:10778000C7D1BAE760681D014019418101330198F2
:10779000D6E71A001B68E6E71325AFE772BD0011B4
:1077A0008644FF1F3866FF1F70BD0011014B187023
:1077B0007047C0468844FF1F14230A0010B51A40C2
:1077C000194204D00122102101F048F810BD4B06E7
:1077D000F9D4012088434000F8E710B514008B0667
:1077E00004D50122102101F039F810BD08230A0048
:1077F0001A40194202D14BB2002B0FDA102101F0CE
:107800002DF8002808D02300F9331B78002BECD08A
:10781000F8342378012BE8D10020E6E7032089071C
:10782000FAD4E2E7F0B51F00184B85B01C68019050
:1078300002910392002C27D1200005B0F0BDA5686D
:107840003301ED186B89019A934211D3029A934246
:107850000ED8002F04D10A9B002B10D12C00EBE78F
:107860003B002978039A6868FEF7F6FC0028F2D1FD
:107870000136B6B2A388B342E1D82468DAE7A36838
:107880000A9A5B891380E9E70026F3E73866FF1F51
:1078900037B50C000A8849880123914217D3002A82
:1078A00015D0651D23792A0002210A48FEF7D4FC71
:1078B000102300280BD023796188208800242A0017
:1078C0000094FFF7AFFF0A23A04200D02300180066
:1078D0003EBDC04672BD001113B50A000888498834
:1078E000012388420BD8002809D0002413790532DF
:1078F0000094FFF797FF0A23A04200D0230018004E
:1079000016BD13B50A0008884988012388420BD8A0
:10791000002809D00024137905320094FFF782FF74
:107920000A23A04200D02300180016BDF0B58BB08A
:1079300003904A8808880E000123824255D300280C
:1079400053D00023012704AC237000227188130058
:107950000092FFF767FF051E3ED02078002835D142
:107960002B78022B18D167706A8983000130E318E5
:1079700080005A8069680222201803F071FE237883
:107980000133DBB22370042B19D93B006889013025
:1079900080B2002BD9D01FE002236370122358431A
:1079A0006A89231804305A8069681022201803F06D
:1079B00057FE23780133DBB22370002BE5D10C4A4C
:1079C0006B899B185A425341DBB2DFE76378012B86
:1079D000E4D12B78022BC7D022780A23002A04D0C6
:1079E00021000398FEF798F9002318000BB0F0BDB2
:1079F0000100FFFF0F4BF0B504001868002816D0F7
:107A000083685D89A54207D88288AE18B44203DA3C
:107A100012019A18934201D10068EFE71E005F89B6
:107A20001036A74204D1002900D00D801800F0BD07
:107A30003300EFE73866FF1F70B505000C000888BB
:107A40000021FFF7D7FF03000120002B04D0220004
:107A50002800197AFFF7C1FE70BDF7B50C000025AC
:107A600001902300F6331B78AB4201D800200AE0D6
:107A70006B00E65A00213000E718FFF7BBFF002833
:107A800002D126800130FEBD017A0198FFF794FEF5
:107A9000002802D03B882380F5E70135EDB2E0E70E
:107AA00010B5040008880021FFF7A4FF030001209F
:107AB000002B03D02000197AFFF77EFE10BD0000D6
:107AC000054B1B68002B01D1180004E09A6852890D
:107AD0008242F6D1988870473866FF1FF0B50E27AE
:107AE000002687B0039302ABFF183E8005001F4BB2
:107AF00040891400984207D02B78013000976A68BB
:107B000080B2FFF78FFE060002212B7818486A68C2
:107B1000FEF7A2FB00280FD06C892000FFF7D0FFF2
:107B2000002802D0013C0419A4B2039B002B00D012
:107B30001C80300007B0F0BD02212B780D486A6828
:107B4000FEF78AFB0028E7D102212B780A486A68F1
:107B5000FEF782FB002807D0002EDED03B88A34230
:107B6000DBD17489013CDFE76C89DEE7FFFF0000B1
:107B700072BD001170BD00116EBD001110B50C007A
:107B8000FFF7DEFC03000220002B0AD0002C00D0FF
:107B900023609B781720FE2B03D00138FF2B00D1E8
:107BA000002010BD73B50D0001A904001600FFF7F9
:107BB000E5FF172805D0002E04D129002000FEF78C
:107BC00027F976BD01221021200000F047FE002891
:107BD000F3D0F6E7014B18607047C0464866FF1FB8
:107BE00037B56B469D1D010004000222280003F0FA
:107BF000B7FC2B88B02B0ED12379122B09D123008F
:107C0000FF339B78012B06D10121608800F0E0F85A
:107C100001E01B2BF8D037BD10B5054B04211870BF
:107C200000F098F8FFF74CFDFEF770FB10BDC04662
:107C30004C66FF1F0020F0B50BB20F0087B08342E7
:107C400034DA274B187803F093FE051E2BD0037807
:107C5000A02B25D103AE3100FEF7E4F8041E0BD1B2
:107C6000B378DB0724D51F4B06341B68002B03D0E9
:107C70003100688898470400A868002801D003F004
:107C800037FD002C08D1184A039B1340174A934232
:107C900006D0B3781B2B03D00121688800F098F838
:107CA000280003F015FF80200002784007B0F0BDE7
:107CB0000F4B1B68002B10D0310068889847041EBA
:107CC000DAD07378002BD7D1B27801A90A704B8033
:107CD0000C716888FDF7F6FFCEE70624F1E7C04691
:107CE0004C66FF1F4466FF1F00FFFF0000011200EB
:107CF0004866FF1FF7B50190822040000D00170075
:107D00001E0003F0FDFB04001320002C12D0B02352
:107D100020002370089BFC22677065802671083064
:107D2000002B08D0190003F09BFC2100019803F000
:107D300007FD0020FEBD089903F0A2FDF5E710B590
:107D4000041E06D00078FD2803D803F0B9FDFF23F8
:107D5000237010BD0A1F93B210B504000220032B3C
:107D600005D882400020024BD1529B189C7010BD58
:107D70006C66FF1F0B8870B5043B04000D000220E9
:107D8000032B0BD80121200000F04CFD0300142030
:107D9000002B03D02900200000F0DEFB70BD0000A6
:107DA00007B51300034A00920A00012100F02CFCE1
:107DB0000EBDC046DD7F001107B50192032200927F
:107DC000024B0A00122100F049FC0EBD5B8000113D
:107DD00007B56B4601AA11800449D880087806339C
:107DE000012802D1190003F09BFC07BD4D66FF1F5F
:107DF0000C4B10B518700023FF210B4A1380138120
:107E000093819380094A53801370517293819372C6
:107E1000D174D3821375517703F0AAFB00F0FCF9FB
:107E200010BDC0467C66FF1F6C66FF1F4E66FF1FBD
:107E3000F0B58DB06B46002003910C229B5E83420F
:107E400000DBB0E05D4B187803F092FD051E00D119
:107E5000A4E00378902B00D09DE006AF0100468897
:107E6000380000F013FA79680400002900D19CE082
:107E70003B88052B6ED13B89032B1CD905AC200018
:107E800000F0A2F86288172A61D83989131D994237
:107E900031D17968237804310291D90738D56078D7
:107EA00000F08EF9071E06D0002303712378012B02
:107EB00008D0132B23D0A868002800D178E003F065
:107EC00017FC75E06288029909A800F0A6F80290F4
:107ED000380000F08BF909AA2378387A0192002241
:107EE00031000092029A00F012F9380000F064F9B3
:107EF000029B002BDFD0300000F080F9DBE7037835
:107F0000032BD8D16288029909A800F0D6F8DEE7E1
:107F1000122B13D1029909A800F0B5F8021EEAD17C
:107F200027498B88002BC6D0887909A9237801912D
:107F300061780091310000F0EAF8BCE7002302AA62
:107F400093833000617809AAFFF72AFFB3E71D4B3E
:107F50000993F6E7042B02D09A1F012AABD8184ADE
:107F6000043B9B00995A0029A5D0D2189078310083
:107F70003A0000F0AEF800289DD13B88042B03D0D6
:107F800001213000FFF724FF012C04D1A86800284C
:107F900001D003F0ADFB280003F09AFD8020039B85
:107FA0000002434018000DB0F0BD012800D182E767
:107FB00001213000FFF70CFFEDE7C0467C66FF1F94
:107FC0006C66FF1F010017000B7803704B7843703D
:107FD000CB788A781B021343438070470A880300DA
:107FE00002700A88120A42700A88012A06D14A8859
:107FF00082704A88120AC2700420704702208242AE
:10800000FBD14A8804309A704A88120ADA708A884A
:108010001A718A88120A5A71EFE710B5040001201C
:1080200082420CD94B780A781B0213432380834287
:1080300006D1CB788A781B0213436380002010BDE1
:10804000022BFBD1CB788A781B02134363804B79D8
:108050000A791B021343A380F0E70B8803700B8897
:108060001B0A43704B8883704B881B0AC3708B8834
:1080700003718B881B0A4371CB888371CB881B0AE1
:10808000C3710820704703000120082A14D14A78E0
:108090000878120202431A80CA78887812020243D2
:1080A0005A804A790879120202439A80CA798879FB
:1080B000120202430020DA80704710B5040001204C
:1080C000022A05D100204B780A781B021343238033
:1080D00010BDF8B5060010200F00150003F010FACF
:1080E00004000120002C0ED0A0230C2229002380A4
:1080F0006780201D002D07D003F0B2FA2100300068
:1081000003F01EFB0020F8BD03F0BAFBF6E7F7B55D
:108110001E00009008AB142017001D78019103F099
:10812000EFF9041E12D0A2230370019B4770438015
:10813000099B057146710C220830002B07D01900ED
:1081400003F08EFA2100009803F0FAFAF7BD0999BE
:1081500003F096FBF6E737B5041E0FD04388002BDB
:108160000CD00025C1881323007A172201950095B1
:10817000FFF7CDFFFF2365806372257037BD0000D8
:1081800010B50C4904004A88002A09D08B89002BBD
:1081900005D00020CB8A0222834201D010BD0122EB
:1081A00013000A20434300204032C854C8184280BC
:1081B0000472F3E74E66FF1F00234380037070478D
:1081C000094B00211A0010B55C88002C06D01C79E0
:1081D000844203D10A234B43D01810BD01310A3326
:1081E0000329F1D10020F8E74E66FF1F10B5040007
:1081F000407A03F065FBFF23637210BD70470430C3
:1082000010B580B203F024FA002803D004214942BB
:1082100003F05EF910BD000070B50025104CA06899
:108220002580A581A580A84202D003F061FAA5604F
:1082300000250C4C0C4B606D1D80230058331D70C5
:10824000A84202D003F054FA656500256068002852
:1082500001D003F04DFA013508340A2DF6D170BD76
:108260001467FF1FB866FF1F0867FF1F70B5041E65
:1082700009D1054D2880A881A880A868002802D0CF
:1082800003F036FAAC6070BD1467FF1FF0B54B8881
:1082900085B00193002343600A7905000F00022A8C
:1082A00000D07BE0CA88032A17D98B685E781978DA
:1082B0003602DC78D8790E4399781B7A24021B02A7
:1082C0000C43034353495BBA0B80331D93421ED1C9
:1082D000042C04D0631F022B0ED9012015E0019A53
:1082E0004D4B1201D35A002B06D00198FFF7BEFF69
:1082F0004A4A1369013313610421B8682E812C8026
:10830000494203F0E5F86860002005B0F0BD434D38
:10831000042C06D0631F022B0FD9EB680133EB60EE
:10832000DBE7019A3C4B1201D35A002B05D0019890
:10833000FFF79CFF2B6901332B61374B3000029311
:10834000019B029A1B010193002301998C468B52D9
:10835000130063449C8003939E81FFF750FF039BAF
:10836000041E986016D00421B868494203F0B0F8A2
:10837000FA880100043A200003F072F90199029A88
:10838000FB888A5A043B9B18029A8B522B68013354
:108390002B60A2E7AB690133AB619EE71E4B0293F2
:1083A000019B1E01029BF35A002B2DD002998C19C0
:1083B000A068002828D0012A26D1FA889B189BB2F1
:1083C0007352A189994217D39B1AC018B96803F058
:1083D00047F9029BA289F35A934200D07DE700221D
:1083E0002B81A3882B80A3686B60029BF2520B4AFF
:1083F00053680133536070E7084A93680133936010
:108400000198FFF733FF68E7044A5369013353616A
:10841000F6E7C0467E66FF1F1467FF1F8466FF1FD6
:1084200070B5051E15D10B4C0B4B1880230058332B
:108430001870606D002802D003F05AF965652500B8
:1084400050356068002801D003F052F90834AC427E
:10845000F7D170BDB866FF1F0867FF1FF0B51700A2
:10846000A12285B0920001934243394B06001B685C
:108470000C009B18D933FF331D78FDF741FF043002
:10848000854204DD3000FDF73BFF0430C5B2BD423C
:1084900007D33A0000213000019B03F011F905B029
:1084A000F0BD2900380002F0F3FF2300C6B25033BC
:1084B0001E700393019B29006365380003F0A8F93F
:1084C000CBB20293002B02D0039B01361E70002614
:1084D0002300503303931B78B34204D8606D002807
:1084E00031D10020DBE7029A2800002A04D0013BAA
:1084F0001000B34200D02800F700E719387003F0ED
:1085000027FA786000280ED03A78019903F0A8F88D
:10851000019A3B780136D3180E4A0193D369F6B21B
:108520000133D361D4E7039B18706065A74205D17E
:10853000084A1320D36A0133D362B0E7606803F0BE
:10854000D7F80834F2E703F0D3F800236365C8E7EF
:108550003409FF1F8466FF1FF7B50D0007000421D3
:10856000686802F0B5FF2B89040003702B891B0A91
:1085700043702B8883702B881B0AC3702E890225B9
:108580000436F6B2FB2E15D81B4B9F4214D10C209B
:1085900002F0B6FF1135011E0CD0902303708E3B04
:1085A0000371043B4380154B8460C680187803F048
:1085B000C7F800252800FEBD5C237B43104AD31872
:1085C0000093583301931B78002B0FD10300320026
:1085D00038000099FFF742FF019B05001B78002B34
:1085E000E8D13800009902F05BFFE3E7054A072570
:1085F000536A01335362DDE7FEFF00007C66FF1F14
:10860000B866FF1F8466FF1FF0B587B00090172083
:108610000F0016000193FFF7F2FD1325041E19D079
:108620000C98031E02D00199201D9847030AE3709D
:10863000052302AAA070043090812770009866700C
:1086400003A993800494FFF787FF051E02D0200042
:1086500003F04EF8280007B0F0BD0000F0B587B079
:108660001F000CAB1B780391059301210DAB060095
:108670001C78049200F0D6F81425002821D02000A0
:10868000FFF77EFD0135041E1BD01149059B0A78BA
:1086900003700132D2B2131EC68001D101231A0029
:1086A0000B7022713000049B03990097FFF7ACFF19
:1086B000051E09D1230021000648074A093302F0AC
:1086C0007FFF280007B0F0BD002363802370F8E728
:1086D0008066FF1F5781001130750000F8B5050056
:1086E0000E00064C064F2368002B02D031002800F4
:1086F00098470434BC42F6D1F8BDC0462467FF1F3A
:108700003867FF1F0123064A5B4253800023137121
:108710005362044A136053609360D36013617047DF
:108720003867FF1F2467FF1F0200002310B50649AA
:108730009C000859002801D1625010BD0133052B5F
:10874000F6D11320F9E7C0462467FF1F034A538878
:10875000181A434258414042104070473867FF1F83
:10876000F0B585B002930AAB1F780CAB1B88009064
:1087700008000E0001920393FFF7E8FF05001120A7
:10878000002D1BD10E48FFF7E1FF04001520002C3F
:1087900014D006220B99A771E01D02F061FF019B26
:1087A00030002371029B29006371009B6680237057
:1087B000039B6562E381FFF791FF280005B0F0BDE0
:1087C000FFFF000010B5FFF7C1FF04000220002CDE
:1087D00012D060880121FFF781FF606A002801D074
:1087E00003F0AEF828220021200003F049F801230D
:1087F00000205B426380207110BD000030B5074A45
:10880000074C5588010013780020A54204D05B1A5C
:1088100059424B415842104030BDC0463867FF1F97
:10882000FFFF0000084A10B501230C00904208D059
:10883000FFF78CFF031E04D0037923405A1E934197
:10884000DBB2180010BDC046FEFF0000024B1879D5
:10885000431E9841C0B270473867FF1F70B50400CF
:108860000D001600FFF772FF002804D10D4B9C424B
:1088700000D0143070BD416A03790520002907D06B
:1088800012221A40102A02D10520002EF2D10F2008
:10889000DB06EFD5897E0C20A94289414942494235
:1088A0000840E7E7FEFF0000030010B5002800D1F4
:1088B00010BD0348034A41889142F9D09847F7E731
:1088C0003867FF1FFFFF0000002330B5C45CCD5C9C
:1088D0006C40D4540133102BF8D130BD0F2300224B
:1088E00010B5C45C64002243CA54C25CD209013B87
:1088F000F7D210BD0200010010B52032103102F095
:1089000097FF10BDF0B58BB00390102005931700B2
:10891000049102F0CDFE0090102002F0C9FE009BF1
:1089200013240190002B05D000280CD113240098AB
:1089300003F006F8019B002B02D0180003F000F8AA
:1089400020000BB0F0BD102002F0B2FE0600102097
:1089500002F0AEFE13240500002E00D1AEE0002888
:1089600019D01022002102F08BFF32002900039859
:1089700002F05EFF041E0ED133787F2B51D83000F9
:108980000099FFF7ABFF009B1B787F2B53D8019911
:108990000098FFF7A3FF300002F0D2FF002D02D0B5
:1089A000280002F0CDFF002CC1D1102002F080FE83
:1089B0000600102002F07CFE0290002E7CD00028E1
:1089C00078D03A000F3223000125121105D00F3361
:1089D0003B4015B25A4253411BB26A1E1201002B92
:1089E00033D0049BD2B298180099029AFFF76CFF1B
:1089F000013D10220021300002F042FFADB2049F81
:108A00002D017D19AF4242D0002C33D0300002F04E
:108A100097FF029B002B00D189E7180002F090FF1E
:108A200085E729003000FFF759FF28002549009A03
:108A3000FFF74AFFA7E729000098FFF74FFF28003C
:108A40002049019AFFF740FFA5E70F210F40049945
:108A50008A18D9B28F4208D9D15C06A819540133BB
:108A6000102BF6D1029A0199C0E7791A4842414188
:108A7000C901F2E73900300006AAFFF725FF3200EE
:108A8000039806A902F0D4FE10370400BAE7002CC0
:108A9000BCD13000029906AAFFF716FF320006A9E2
:108AA000039802F0C5FE082204003100059802F088
:108AB000D7FDABE71324A9E71324AAE7002800D0C9
:108AC0006EE733E778BD0011F0B58BB00F001600EC
:108AD0000225009000283FD0002A3DD00B1DDBB2BC
:108AE0001800029302F0E4FD1135041E34D0FDF7A6
:108AF00047FD05003A000099201D02F0A1FFEBB2EE
:108B00000393E3702B0CDBB22F0A00936370FFB268
:108B10002B0E2370A7700193FDF72CFD102201008E
:108B200006A802F08DFF2100029A04AB06A8FFF709
:108B3000E9FE051E0DD1039B08223370009B04A99A
:108B4000B370019B7770F370301D02F079FFFDF771
:108B50001DFD200002F0F4FE28000BB0F0BDF0B5C2
:108B60008FB00D00149E039004920593002A03D148
:108B7000022420000FB0F0BD002EF9D00398FFF7BB
:108B8000E5FD1424071EF4D07278337812021A43DC
:108B9000B3781B041343F27812061A43036A019256
:108BA000934201D30133E3D1002D03D03B7901245B
:108BB0009B07DED50822002106A802F061FE059B76
:108BC00013240433DBB21800029302F071FD051E7A
:108BD000CFD0059A0499043002F032FF042231000C
:108BE000280002F02DFF3900102210310AA802F0EF
:108BF00027FF2900029A06AB0AA8FFF783FE041E8E
:108C00000FD1082206A908A802F01AFF0822311D78
:108C100008A802F0DDFE012807D101990398FDF7AD
:108C2000C9FC280002F08CFEA3E70124F9E700004C
:108C300070B51C4C05002368181E10D0002D14D1EF
:108C40001A78002A0CD1981C083202F009FD02F0B3
:108C50009FFD0135002808D123681D70012070BDDB
:108C60000A331800082202F0FBFC2368002BF5D021
:108C7000122002F045FC061E0DD0C12321680370AE
:108C8000457002311022023002F0EAFC2368310004
:108C9000587802F055FD206802F052FE0023236050
:108CA000DCE7C0466067FF1FF8B504002020FDF731
:108CB00055FB0D4EA700BB590500002B0DD0002819
:108CC0000BD0D878FF2809D108492A000C55F35950
:108CD00007480333611802F073FCF8BD290002F065
:108CE000C7FD0028F0D1F8E77C67FF1F6467FF1F0E
:108CF000019F001170B5064D84006359002B05D00B
:108D0000D87802F0DDFDFF226359DA7070BDC046ED
:108D10007C67FF1F70B506008CB00C0015000021A9
:108D20003022684602F0ACFD31001022684602F0A5
:108D300087FE1D2021000322684402F081FE684660
:108D4000FFF7D8FD2D21040003222800694402F01A
:108D500077FE20000CB070BDF0B50700160097B08C
:108D600001931CAB1D7830221EAB00910AA8002194
:108D70001C7802F085FD102239000AA802F060FE7E
:108D80001022002102A802F07BFD0722310002A878
:108D900002F056FE072202AB9818631E9C4101990F
:108DA00002F04EFE02AB9C732B005A1E934102AAA6
:108DB000D3730021102206A802F062FD06221D993D
:108DC00007A802F03DFE1A2002ABC01806221F9928
:108DD00002F036FE102200990EA802F031FE102299
:108DE00002AB0EA908781C78013A6040D2B2087034
:108DF00001330131002AF5D10AA8FFF77BFD1022CB
:108E000012A904000EA802F02BFC102206AB0EA93A
:108E100008781D78013A6840D2B2087001330131F8
:108E2000002AF5D10AA8FFF765FD04431022209817
:108E3000E4B212A902F004FE200017B0F0BD70B534
:108E40000E0014008CB00100102268461D0002F0D4
:108E5000F7FD3100082204A802F0F2FD21000822EB
:108E600006A802F0EDFD6846FFF744FD040010225D
:108E7000280008A902F0E4FD20000CB070BDF8B590
:108E800006000D0000243719AC4200D3F8BD02F0F3
:108E9000DFFD030A3B70631CDBB201379D4203D93F
:108EA0000234F054E4B2EEE71C00EDE773B50600BF
:108EB0000C000225002819D0002917D0032101A891
:108EC000FFF7DDFF6B469A793F231A4001331343C6
:108ED0006A463000937101A92200FFF71BFF051EAF
:108EE00004D10322E01C01A902F0BAFB280076BDE0
:108EF00003785807DA08C00FD20080009B071043A0
:108F00009B0F1843C0B2704707230B40C908C90024
:108F10000B4303707047000070B50400FFF7EAFED2
:108F2000134DA4006359002B21D0186A002801D0EA
:108F300002F006FD2B59986E002801D002F000FDCA
:108F40002B59D86E002801D002F0FAFC2B59186F6B
:108F5000002801D002F0F4FC2B59586F002801D0F2
:108F600002F0EEFC285902F0EBFC00232B5170BDFF
:108F70007C67FF1F0E4B8000C35870B50C00002BA0
:108F80000FD09D68002D0CD02B78201D0B706B78B6
:108F90004B70A97CFFF7B8FF2B7E23726B69E360EF
:108FA00070BD10220021200002F06AFCF8E7C046E4
:108FB0007C67FF1F014B18607047C0467867FF1F32
:108FC000074A03008000825810B5002A06D0D088D6
:108FD000984203D1012901D1FFF79EFF10BDC04681
:108FE0007C67FF1FF0B5264E95B087000B93BB59E9
:108FF0000500099112200A92002B31D0D888FFF782
:10900000A5FB04001420002C2AD0280010A9FFF78B
:10901000B1FFBB591E781D6A002E23D00895FDF7BD
:10902000EFFA07000020FDF7F1FA0790A379E61D9B
:10903000069310AD0CA9089800F0E2FA0EA92800DA
:1090400000F0D7FA0B9B0A990493069B09980293A8
:10905000079B0396019300970EAB0CAAFFF77CFECB
:1090600015B0F0BDFDF7CCFA06903000FDF7CEFA52
:10907000E31DA779079310AB06000893DAE7C04613
:109080007C67FF1F30B50C4C85002A59030085B062
:109090000120002A0ED018006946FFF76BFF2B59FC
:1090A0001A78D888054B002A00D1054B6A4607215B
:1090B00000F0D9FB05B030BD7C67FF1FF3950011B0
:1090C0000196001130B5094C8500295985B0102250
:1090D0006846253102F0C4FA2A591121044BD08880
:1090E0006A4600F0C0FB05B030BDC0467C67FF1F7C
:1090F0009D96001130B5094C8500295985B0102284
:109100006846353102F0ACFA2A591121044BD08857
:109110006A4600F0A8FB05B030BDC0467C67FF1F63
:10912000DB960011F7B54D4F86001020F4590D0065
:1091300002F0BEFAF3592062186A132200286CD09C
:10914000033A29009C6802F08BFAF3591A780192CD
:10915000002A58D11E6A227D317B9446514001225B
:10916000019F114201D167461740217D9143394348
:109170002175377B4F40BC4660460027800701D4ED
:109180004F081740012102208F40227D82433A433D
:109190002275377B5740BC4660460027400701D404
:1091A00097080F400420227DBF0082433A43227576
:1091B000627D002794466046727B42400A4201D19C
:1091C00067460F400121627D8A433A436275777B8F
:1091D0005740BC4660460027800701D457080F401F
:1091E0000220627D7F00824317436775767B0022F1
:1091F0007E40760701D4BA080A400426617D9200B9
:10920000B1430A4362756A78002A08D06278002A5E
:1092100005D005220533DA7700221000FEBD0422B6
:109220002979114205D1A17C114202D10533033ABB
:10923000F1E7019A21782C78002A02D10A00210056
:10924000140018220429E8D8042CE6D8052060432D
:10925000034A05331218525CDDE7C0467C67FF1FE6
:1092600088BD001110B50A001121024B00F0FBFA75
:1092700010BDC046379700110B0030B587B001AD67
:109280002B806B4604001100981D082202F0E8F9BB
:109290002A000B212000024B00F0E5FA07B030BD98
:1092A0005F97001110B50A001121024B00F0DBFAA4
:1092B00010BDC046B397001113B50B0011006A46EC
:1092C00013706B4604000622581C02F0C9F96A4666
:1092D00008212000014B00F0C6FA13BDD3970011FE
:1092E00010B50A001121024B00F0BDFA10BDC046B6
:1092F000239800117FB505000B4BAA00D458080035
:10930000002C0FD0666F237FE28821780396266FAA
:109310000296E66E0196A46E0094FDF709FC280003
:10932000FFF7FAFD7FBDC0467C67FF1F10B5172110
:10933000FFF7E0FF10BD000070B50A000D00064BFE
:109340000221040000F08FFA060029782000FFF7C0
:10935000D1FF300070BDC0460397001170B586B0D4
:1093600000236A461370836804001D78681E0A286B
:1093700059D801A902F03CFB060633373B3F43476F
:109380004B4F5300180000F042F9062312284BD02F
:1093900000281BD16088FFF7D9F90823002813D0D3
:1093A0004279002A47D1264B1A78072312070BD59A
:1093B000244B1A680723002A06D01668002E03D013
:1093C000290001AAB04703006A4613706B461B7858
:1093D0006088002B2AD1FFF767FC06B070BD18002B
:1093E00000F06CF9D4E7180000F087F9D0E7180016
:1093F00000F093F9CCE7180000F0ADF9C8E71800C9
:1094000000F0C3F9C4E7180000F0F6F9C0E718004F
:1094100000F0F6F9BCE7180000F013FAB8E71800FE
:1094200000F013FAB4E707236A46137069466088B0
:10943000FFF782FFD1E70523012AC5D1024BB8E728
:109440000966FF1F7467FF1F7867FF1FF8B52C4F71
:109450008600F35904000D00002B40D0DA888242C8
:109460003DD15A78062A33D11A78002A2ED001200D
:1094700099681A6A097D014206D0157B054203D01E
:1094800007225A700120F8BD0220014204D0157B4A
:10949000054201D00922F4E70420014204D0127BE6
:1094A000024201D00B22ECE7164B1B68002BE9D0DF
:1094B0005B68002BE6D020009847BB5900215B7801
:1094C000122BDFD12000FFF715FFDBE70E4BECE797
:1094D000112A04D1002900D032252900F2E7002DFD
:1094E00008D12000FFF732F9002803D010230279B9
:1094F0001343037121002800FDF798FAC2E7C04624
:109500007C67FF1F7467FF1F7867FF1F70B50E4EE3
:109510008500AB590400002B13D01B78002B11D110
:109520000A4B1B68002B04D05B68002B01D0200085
:10953000984773595B78122B03D100212000FFF765
:10954000D9FE70BD024BECE77C67FF1F7867FF1FF9
:109550007467FF1F094B8000C3581020002B0CD0EC
:109560001A6A002A09D09B68002B06D0127A1B7E4B
:10957000101C9A4200D9181CC0B270477C67FF1FAC
:1095800070B503000D0014000220002A30D000291D
:109590002ED013700B78081D53704B789370FFF723
:1095A000A7FCE070012002212B7A23716B7B034022
:1095B00063716A7B0A401343042263716E7B164019
:1095C000334363716E7BF608F600334363712B7B84
:1095D0000340A371287B014000200B43A371297B2A
:1095E0000A401343A3712A7BD208D2001343A3710C
:1095F00070BD10B50A0001000120FFF7C1FF10BDCA
:1096000010B50A0001000220FFF7BAFF10BD70B5C7
:1096100006000C000220002E30D000292ED07378D6
:10962000201D0B70B3784B70F178FFF76DFC0122B1
:109630003579257271794B10080013409340104022
:109640000343881010408000C9080343C9000B433E
:109650006373B1794B1008001340934010400343EB
:10966000881002409200C9081343C9000B4321200F
:109670002373FCF773FE854201D2122070BD2220B5
:10968000257AFCF76BFE8542F7D823781820042B47
:10969000F4D86378012BF1D80020EFE7030010B570
:1096A0000220002909D0002B07D00322481C0A7091
:1096B00019000D3201F0D4FF002010BD030002227A
:1096C000080010B5002B06D0002904D00E32591C1A
:1096D00001F0C6FF0022100010BD030010B50220EB
:1096E000002909D0002B07D00422481C0A70190059
:1096F0000C3201F0B5FF002010BD10B5FFF7DEFF02
:1097000010BD03000220002906D0002B04D0052242
:1097100000200A701B784B70704703000220002B5A
:1097200008D0002906D05B7800200B70013B082B85
:1097300000D918307047030010B50220002909D065
:10974000002B07D00622481C0A7019000A3201F0CB
:1097500087FF002010BD10B5FFF7B0FF10BD02005D
:109760000B00022010B500290ED0002A0CD00721D2
:109770001970118859701188090A997011180822F6
:10978000D81C01F06DFF002010BD03000A0002206C
:1097900010B5002B0CD000290AD09978587809020E
:1097A00001431180901CD91C082201F059FF0020B0
:1097B00010BD030010B50220002909D0002B07D0EE
:1097C0000822481C0A701900921801F049FF002075
:1097D00010BD02000B00022010B500290BD0002A9A
:1097E00009D009211970117818185970511C0622D6
:1097F00001F036FF002010BD10B5FFF75FFF10BD70
:1098000002000B00022010B5002A09D0002907D061
:109810005178197011180622581C01F021FF002000
:1098200010BD030010B50220002909D0002B07D07D
:109830000A22481C0A701900063201F011FF0020AC
:1098400010BD10B5FFF73AFF10BD02000B0002205B
:1098500010B5002A06D0002904D018005178FFF76F
:1098600053FB002010BDF0B585B017001E006A46FE
:1098700006230500080091819380FEF7C0FC1324A5
:10988000011E02900CD03800B047041E05D12800FC
:1098900001A9FEF76FFA041E02D0029801F028FF1A
:1098A0002800FFF701FA200005B0F0BDF0B5040074
:1098B0008BB0019115000021102202A801F0E0FFF9
:1098C000334EA700B85900283CD0C388A34239D1F1
:1098D0000378002B36D14278062A18D10200010005
:1098E000553235310C3006ABFFF7A9FA002829D1E3
:1098F0002000FFF72FFE020006A902A801F0B0FE2B
:10990000200002A901F09CFF01200BB0F0BD816E88
:10991000002917D00B8A112A28D19D420ED1019817
:109920001231093A02F054F8012807D1BB5920003E
:109930009D6EFFF70FFE29000200DEE732212000B6
:10994000FFF7D8FC2000FEF701FF061E1BD0416A7E
:10995000002918D00B8AAB4215D108220198123188
:1099600002F036F801280ED1716A0AE09D42E9D171
:1099700008220198123102F02BF80128E2D1BB59DC
:10998000996E8A7EB9E7200001F0CAFDBCE7C046A7
:109990007C67FF1FF0B56B4D87007E5985B033782B
:1099A00002900393002B00D087E0B368346A0193E0
:1099B0007078062817D101221B7D134202D0217B2B
:1099C000114218D10222134202D0217B114251D1FF
:1099D0000422134203D0237B134200D08BE0019B6F
:1099E0005A7DEB5991E007380428F8D802F000F8C6
:1099F000032E42678300B36E002B03D11C2001F0BD
:109A000057FEB066EB599C6E002C1CD01022002132
:109A1000200001F035FF0298FFF79CFD01002000B7
:109A2000FFF72DFA02F014F82082200008211230EE
:109A3000FFF725FA0298FFF78DFDA076EB5921007C
:109A4000D888FFF70FFC0822EB591CE0B36E002BFF
:109A500005D01A00198AF0881232FFF70DFC022295
:109A6000019B197DEB5911423DD0207B10423AD029
:109A7000073208E0F488FCF7DBFD01002000FFF767
:109A800011FC0A22EB595A70029B9C002A59537808
:109A9000073B042B11D8D088FEF758FE00284ED083
:109AA000C3895A08D2182849029B0298CB542B59D3
:109AB00041180433254801F083FD05B0F0BDFCF7E3
:109AC0009FFD03000120834201D100200393EB5945
:109AD000DE88FCF79BFD039902003000FFF7ECFBEA
:109AE000019AEB59117D042211420CD0217B1142C5
:109AF00009D00B22C7E7F688FCF73CFD01003000D7
:109B0000FFF7EEFB6BE7019A527D01210A4204D078
:109B1000607B084201D00C22B5E702210A4204D042
:109B2000607B084201D00E22ADE704210A4204D036
:109B3000627B0A4201D01022A5E71222A3E7FA2293
:109B40005200B0E77C67FF1F8067FF1F0B9F00116B
:109B500010B5064B1A780423100018401A4200D0A2
:109B60000348FFF727FA002010BDC0460966FF1F13
:109B70008C44FF1F70B50400FFF7D4FA051E43D1D3
:109B80002000FFF77FFA234EA400A0598268937C3F
:109B9000DB0708D50321036A1B790B40012B02D197
:109BA000017F0B430377431DD97F8B1E022B0DD8FA
:109BB000022900D00121C088FCF790FF042133590D
:109BC0001A7F59700A431A77280070BD01290CD1F9
:109BD00002231022437000210C3001F051FE305955
:109BE00010213530FFF74BF9EEE70529ECD10223C0
:109BF000D118437010220C3001F032FD0423325989
:109C0000117F0B431377EAE708251828DCD1053DBF
:109C1000DAE7C0467C67FF1FF0B58BB0059143883B
:109C20007E4F9E00F45915000493002C15D1012994
:109C300002D000200BB0F0BD101D57781678FFF74A
:109C400057F9EB68320002932B7A04990193009044
:109C50003B002000FCF70CFFEBE7E388049A9342FB
:109C600001D00820E6E72378012B00D1D4E0059B42
:109C7000581E092800D9CFE001F0BAFE05CE0A2906
:109C8000CC506C859AB229000498FFF773FFD1E796
:109C9000200029001022453001F0E2FCB9594B7830
:109CA000042B02D1013B4B70C3E70B000A002533A4
:109CB00035320C310498FFF795F90498FFF702FA52
:109CC0000522431E9841BB59C0005A70B2E72000DC
:109CD00029001022553001F0C3FC049B4F4C9D001D
:109CE000295904980A0006AB55320C31FFF77AF96E
:109CF00029591022453106A801F06AFE012808D131
:109D00000498FFF7F7F90590002804D106222B5993
:109D10005A7005988EE708230593FAE763780C2BB1
:109D20007AD1E36E002B03D11C2001F0C1FCE06668
:109D3000BB59D86E00286FD01022290001F090FC8A
:109D4000BB590498DC6EFFF705FC0D22A076BB59C9
:109D50005A706EE7E06E00285ED063780D2B5BD101
:109D60002B8808220382A91C123001F079FCBB5910
:109D70009A68517D0222114226D0186A407B104217
:109D800022D00C32E4E763780E2B45D1236F002BF1
:109D900003D1162001F08CFC2067BB59186F0028F6
:109DA00003D01022290001F05BFC0F22BB59CFE742
:109DB00063780F2B30D1206F0622691C103001F020
:109DC0004FFCBB599A68517D0422114203D0196A95
:109DD000497B1142D5D100210498FFF78BFA28E77F
:109DE000636F002B0DD0BB59586F0028F3D01022A1
:109DF000290001F035FC0122BB5952425B6F1A6108
:109E0000E9E7142001F054FCBB5960675B6F002B3D
:109E1000E9D126E72978DFE707200BE77C67FF1FFA
:109E200010B5064C207001F05BFC06212078FDF790
:109E300091FF0348FEF778FC10BDC0468F67FF1FF7
:109E4000C18F001100200BB270B50D00834216DAED
:109E5000264B187801F08CFD041E0DD00378922B50
:109E60000ED0A02B37D0224B1878FF283AD02100F3
:109E700001F066FC002835D180200002684070BDEA
:109E800043780E2B0BD03E2BEDD18378052B12D0CF
:109E9000082BE8D181798088FFF7D8FA08E0154BC4
:109EA00082889A42DFD183681878591CFEF7C0FE79
:109EB000002817D1D7E7104B1B785B0712D50F4B43
:109EC0001B68002B0ED09B68002B0BD0C289811D14
:109ED00080889847ECE7FFF741FAA068002801D096
:109EE00001F006FC200001F0F3FDC5E78F67FF1FBE
:109EF0008544FF1F182000000966FF1F7867FF1FB9
:109F000010B50078FFF712FA10BD10B50078FFF712
:109F1000FDFA10BD0C234343084A10B59B185A683C
:109F2000002A03D0012901D1904710BD9B68002B66
:109F3000FBD00029F9D19847F7E7C046AC67FF1F6F
:109F400010B5162813D801238340094A946B1C438B
:109F50009463506B98435063D46B2000984301295D
:109F600001D120001843D063116B0B43136310BD64
:109F700000800040F0B500240127154B85B0DA6B56
:109F8000144E03921A6C0192DA64019BE3403B4247
:109F900017D0039DE5403D400295E5B202992800A7
:109FA000FFF7B8FF316A736A002908D03900002B27
:109FB00001D0029979402800FFF7C2FF01E0002B91
:109FC000F9D101340C36172CDFD105B0F0BDC046F5
:109FD000008000409067FF1F10B5012402002000A0
:109FE000162A08D8054B5968D140214204D0186878
:109FF000D0400123184010BD186DF9E700800040E3
:10A00000162807D80122064B8240002903D0D968C0
:10A010000A43DA607047D9689143D960FAE7C046CD
:10A020000038004030B5162818D8032444430F4B9D
:10A03000E25C1B199C785D7801232D1B0135AB4038
:10A04000013BA340A140DB430C00122807D808497C
:10A0500092005218116819402143116030BD054A21
:10A0600011680B4023431360F8E7C046CFBD0011D1
:10A0700008F0004014F00040C21F70B5D4B20623AF
:10A08000092C0BD80125084C9540002908D0002147
:10A09000FFF7C8FF23682B4323600023180070BD1F
:10A0A0002368AB43F8E7C04600380040F0B51628F7
:10A0B00026D8214B1B185B78022B21D10324444363
:10A0C0001E4A1F4EA35C1219947801221500854088
:10A0D000B76B013CE4B23D43A240B563194C122872
:10A0E00015D89B0000290CD117495B1899680A43C1
:10A0F0009A600123205C154A834011680B4313606A
:10A10000F0BD11495B18996891439960F1E70E4BD6
:10A1100000290DD159690A435A61225C1328E8D0FD
:10A120000123203A93400A49086803430B60E7E79C
:10A13000596991435961F0E79067FF1FCFBD001146
:10A140000080004014BE001100F00040A0F000406C
:10A15000A4F00040F8B500241B4E1C4D1C4B1B5DA9
:10A16000012B1FD1184A9269E2401A420BD00122FA
:10A17000AA5693402200143AD2B2022A09D81549AD
:10A180004A6913434B6101340C360235172CE5D173
:10A19000F8BD0022AA560F499200521891680B434D
:10A1A0009360F0E7022BEED1E7B23800FFF714FF1F
:10A1B00001235840C1B23800FFF778FF3800FFF79D
:10A1C0000BFF7077DFE7C0469067FF1FA1BD00114E
:10A1D0009167FF1F00F00040012202388240054BCA
:10A1E000002903D059690A435A617047596991435C
:10A1F0005961FAE70038004070B504000D000520F1
:10A20000162C1AD800212000FFF7FAFEA31E012BFE
:10A2100003D801212000FFF7DFFF00212000FFF716
:10A220002BFF01220A49A2400A4B4868012D05D1A3
:10A2300002431B194A605D70002070BD9043486066
:10A2400002211C196170996991439961F4E7C04634
:10A25000008000409067FF1F10B516280AD8012221
:10A26000074B8240002906D019680A431A60012171
:10A27000FFF7C2FF10BD196891431960F7E7C046A8
:10A280000080004070B505000520162D17D80C235E
:10A2900000246B430A4A21009B181C70094B2800BC
:10A2A0005B195C70FFF7A8FF0123AB402000064953
:10A2B0000A681A430A6005490A689A430A6070BD31
:10A2C000AC67FF1F9067FF1F348000403080004064
:10A2D00070B504000E00FF2813D003250540FFF7DA
:10A2E000D1FF084AA3089B009B183F22ED00AA401B
:10A2F000AE40196820009143314319600121FFF7F6
:10A300007FFE70BD18380040F8B505000520162DF9
:10A3100025D80C246C43124BE4186368002B03D13E
:10A32000A3680D30002B1AD0022201270D4B00210B
:10A330005B195A7028002770FFF75EFF63681E1EC6
:10A3400008D0A3683E00002B04D02800FFF744FE8D
:10A350004640F6B228003100FFF7F2FD0020F8BDBC
:10A36000AC67FF1F9067FF1FF7B5C420FF222B4B80
:10A3700080001958002491437F3A0A431A508022E2
:10A38000274F5202274E1A60274B1D5D002D21D00A
:10A39000A31E012B03D80121E0B2FFF71DFF012D01
:10A3A00018D11F4B9B69E3402B4213D0E3B2180036
:10A3B0000193FFF711FE01000198FFF74DFFE3B293
:10A3C000143B022B1DD801217156184A8D40536948
:10A3D000AB4353613B7F002B0DD0E5B22800FFF764
:10A3E00093FF2800FFF7F8FD7B7F0100834202D036
:10A3F0002800FFF78FFD01340C370236172CC3D12C
:10A40000F7BD012100237156F3568D40074A9B008A
:10A410009B189A68AA439A60DCE7C04600E100E016
:10A420009067FF1FA1BD00119167FF1F00F0004062
:10A4300010B504000520162C0CD801212000FFF7D0
:10A44000DBFE0123044A002011194B70A3409169DF
:10A450000B43936110BDC0469067FF1F70B50E009F
:10A4600015000400FFF70EFF0C236343094A200088
:10A470009B189D605E60FFF747FFF021064B074A7F
:10A480008900051E5A5002D02000FFF7FBFE28006D
:10A4900070BDC046AC67FF1F0000FF1F759F001115
:10A4A00070B5134D07202C78002C1FD19822210065
:10A4B0005200280001F094F90123C420FF222B70E0
:10A4C0000C4B80001C635C630B4B1C605C600B4B93
:10A4D000195891437F3A0A431A50802252021A6057
:10A4E0000D20074A074901F093F8200070BDC046CF
:10A4F0009067FF1F00800040A0F0004000E100E0F6
:10A5000069A3001155A10011030010B50620072B07
:10A5100009D8054A137001F02BF9D7210020034B0D
:10A52000034A89005A5010BDB444FF1F0000FF1FAA
:10A53000151BFF1F70B51D0002240C2910D8094AF5
:10A54000CA40D2070CD5FBF715FF041E08D1059AA7
:10A5500004992800FBF72AFFFCF798FDFFF7F8FAAB
:10A56000200070BD1210000030B50D7802232C00C1
:10A570009C43184201D02B431C0008252300AB4309
:10A58000284201D02B00234320241D00A543204254
:10A5900001D01C4325002A230D70184204D01178E5
:10A5A0001E3B0B43137030BD0028FCD10C211378E7
:10A5B0008B43F7E7F8B51D0006AB1B88140007AA0C
:10A5C0000E000B201778002B27D10A78022A49D1D8
:10A5D0004A68507811780002244A084380180428F9
:10A5E00040D801F005FA03121D1B2300F06800F0AB
:10A5F00037FF021CC0B2B84200D93A1CD2B22000C8
:10A60000F1682A8001F02CF806E00222F3681B882A
:10A610002A8023701B0A63700020F8BD0622EEE733
:10A6200001232B80F3681B782370F5E7F368002B78
:10A6300016D008222A801A8822701A88120A62709C
:10A640005A88A2705A88120AE2709A8822719A88EF
:10A65000120A6271DA88A271DB881B0AE371DBE7F8
:10A660002B80D9E701202B80D7E7C04600D6FFFF1B
:10A67000F7B516000A781D0008AB1F880C000123EF
:10A68000022A18D14A685078117800022B4A0843F0
:10A69000801803280FD801F0ABF902254439E0688F
:10A6A00000F0DEFEC0B20723B84204D37B19019349
:10A6B000152B02DD0D231800FEBDE0682A003100D5
:10A6C000C01900F0CDFF6B4600209B88E268D05493
:10A6D0001B4B1B68834203D01B68834200D0984702
:10A6E0000023E8E70B23002FE5D1022DE2D1737898
:10A6F00032781B021343E2681380114B1B68002B56
:10A70000EED01B68002BEBD00120E8E70B23002FD5
:10A71000D1D1062DCED12A003100E06800F0A0FF93
:10A72000DEE70B23002FC6D1012DC3D1327875335C
:10A73000012AC0D8E3681A70D2E7C04600D6FFFFEE
:10A740009C69FF1F70B50C001500072837D801F071
:10A750004FF9041436361B36242E182015290BD831
:10A76000184E16220021300001F08AF8220029003C
:10A77000300000F075FF002070BD18200229FBD1C9
:10A780001288114B1A80F6E718200829F4D10A0024
:10A790000E48290000F0E4FEEDE718200129EBD176
:10A7A0000B4B10780B49DA69FFF7DEFEE3E7182060
:10A7B0000129E1D1064B10780749DA6BF4E7022052
:10A7C000DAE7C0468469FF1F3245FF1F2845FF1F97
:10A7D000B844FF1FE044FF1F0045FF1F030010B5F2
:10A7E0000020DB0704D50721024A034800F08CF85B
:10A7F00010BDC0462CBE0011B844FF1F054A03001F
:10A800001068002803D082889A4201D1806870477E
:10A810000068F6E7A06BFF1F0A88030008009A4251
:10A8200004D08A8804309A4200D00020704700008B
:10A83000F8B5F82200230D4F0D4E7968050042430C
:10A840003370994200D07B600A4C0021200001F057
:10A8500017F800231A007C60AB4202D1002033704D
:10A86000F8BD01332280DBB2F834F5E7A06CFF1F9E
:10A870009C6CFF1FA46BFF1F73B56B460190060015
:10A88000684615001980FCF733FF041E11D1002D16
:10A890000FD07689002E11D00C2000F009FF00287F
:10A8A0000ED0084A0460136886808560002B02D1B0
:10A8B0001060200076BD1A001B68F7E70224F8E755
:10A8C0001324F6E7A06BFF1F012100220A4B10B5ED
:10A8D00049420A4C198099809A719A70084B2070ED
:10A8E000012019805A60FFF7A3FF2078FCF75EFF74
:10A8F0000448FDF719FF10BDA469FF1FA86CFF1FD6
:10A90000A06CFF1FB5A90011022310B5002802D0CA
:10A91000FFF7B2FF0300180010BD0000030010B5E0
:10A920000020DB0704D50421024A0348FFF7A4FFF7
:10A9300010BDC04640BE00113845FF1FF0B50E26C1
:10A9400087B003930CAB1F8802ABF6180500080014
:10A9500031000292FDF74EF804000120002C0FD0C8
:10A960003088FFF74BFF03000E20002B08D05E68F5
:10A97000002E05D021002800039B029A0097B047C3
:10A9800007B0F0BD0A4B10B5984207D10122002351
:10A9900052420A808B708A808B7110BDFFF73CFF9A
:10A9A0000028FAD001235B42038000238370F4E780
:10A9B000FFFF0000F8B5050001290AD1134E00245D
:10A9C0003388F827AB4219D028001149FFF7DAFF86
:10A9D00006E0022904D10139FDF724FF0028EDD05B
:10A9E000F8BD3B0063437268D018D35A002B09D0DE
:10A9F0003A00002100F044FF0134E4B2054B1B781B
:10AA0000A342EED801235B423380DDE7A06CFF1F39
:10AA1000A469FF1F9C6CFF1F10B5FFF7FDFE03002C
:10AA20000020834200D0987810BD0000F0B589B0B6
:10AA30001C000EAB80CB03901E8810AB1B780492D9
:10AA400002930B7A0D00DB0616D42B780593022BAC
:10AA500024D00498FFF7D2FE002812D003689C4649
:10AA6000002B0ED0029B2200019329003B0064467C
:10AA700003980096A04705E00498FFF7BFFE002862
:10AA800002D10E2009B0F0BD8368002BF9D00A2254
:10AA90002900039898470028D7D0F3E76B685878C7
:10AAA0001A786B4B000210439842D2D8043B98426C
:10AAB00010D2684B984242D015D8674BC018012875
:10AAC000C7D80B20002EDDD1EB681A7859683A8080
:10AAD000200028E0614BC018032800D979E000F07D
:10AAE00087FF846A789E5E4B9842B2D10B20002E7D
:10AAF000C8D101233B80EB6831001B782370688943
:10AB0000013080B2FCF776FF3A88031E0ED0017840
:10AB100002328A183A80428962704289120AA2700F
:10AB200059680278E01C00F09BFD06E004323A8090
:10AB300031000422601C00F0A3FE0020A2E70B20DD
:10AB4000002E9FD1EB6807A91E8804233B80330A9F
:10AB5000300026706370FCF74DFF051E28D004AB53
:10AB60009A890E2304A95B183E49C668FCF7B6FF14
:10AB700000280BD12B783C486A680599FBF76CFBE1
:10AB8000002803D1012304AA5B42D3813278022A30
:10AB900006D17168201D00F063FD3B8802333B80C5
:10ABA0000E2304AA9B181B88A3701B0AE370C4E73A
:10ABB00004ABDE81F4E70B20002E00D062E7E968E9
:10ABC0000398FFF729FF02233B802070000A607082
:10ABD000B3E70B20002E00D054E70222EB681B885D
:10ABE0003A8023701B0A6370A7E7E86800F038FC1E
:10ABF000C2B203000720B24200D243E70DD002994F
:10AC0000DBB27118994202DB921BD3B20293029B12
:10AC1000E9681A003B8089195AE70023F6E70B2000
:10AC2000002E00D02EE70722EB683A801A782270B7
:10AC30005A7862705A88A2705A88120AE2701A7999
:10AC40002271DA886271DB881B0AA37175E7C0463E
:10AC5000042900000228000000D8FFFFFFD6FFFFF4
:10AC600003280000FFFF000070BD0011F0B58DB09B
:10AC70006B460020089120229B5E83423DDAA64B62
:10AC8000187800F075FE071E32D00378B02B2CD157
:10AC90000079023816281FD800F062FD17001E0048
:10ACA0001E001E0031001E0096001E001D011E0029
:10ACB00052011E0073011E00CD011E0050021E0035
:10ACC0001E001E008E021E00E302944B94491B8856
:10ACD00078880B80FBF700F83800FCF781FF914B78
:10ACE0001B68002B01D038009847380000F0F0FEB8
:10ACF0008020089B0002434018000DB0F0BDF622F2
:10AD00000021874800F0BCFD0BAA3B7B798938897C
:10AD100000923A000D32FCF785FD0400804B1B7851
:10AD2000002C3FD146E0804B788805937F4B410053
:10AD3000CB5A0BAE073BDBB2328802930023019360
:10AD40007B4B210006930093059BFFF76FFE744D2C
:10AD5000002810D1069B3A8A1B889A420BD13800F2
:10AD60000599123000F034FE002804D02B78628957
:10AD70009B00EB185A80162306A81B183288200067
:10AD80007989FCF7ABFE2B7804009A00AA18518849
:10AD90000029C3D00133DBB22B70002807D006A9ED
:10ADA000C98A9180634A12889A42BCD802E0012184
:10ADB00049429180002B04D059497888FAF7C0FFA6
:10ADC0008AE73E890A2479E000253E89574B06939D
:10ADD0007B88069A5B009B5A033B9D4202DB002D59
:10ADE000F0D05BE0162206A812183B7B798900920E
:10ADF0003A0030000D32FCF715FD0590002858D0C0
:10AE00004689017A7888FCF7D7FC041E44D1464B6A
:10AE100078880793069B4100C95A454B0439C9B24B
:10AE200006AAD28A06930291019400930599079B82
:10AE3000FFF7FCFD041E2FD1069B39491A88931C8D
:10AE4000002D26D14B807988384B4900CB5A5119B7
:10AE5000033B8B4220DD059B31485B8941190B7117
:10AE6000A91C0135C9B2EDB2059145191B0A2B7118
:10AE7000059B2D490433181800F0F2FB2C4B059A62
:10AE80001B88D318DDB22C4B9E4205D00136B6B2DA
:10AE90009CE749889942D6D0002D0CD0204C280040
:10AEA000618800F0BDFB207021007888FAF758FF18
:10AEB00012E7059CF0E7002C00D183E77B78142B88
:10AEC00000D109E716493B794E800B700C717888E8
:10AED000FAF7F8FE00E7162406ABE41821003889DB
:10AEE000FCF788FD011E00D1B7E1788822880F4C5D
:10AEF00045002C5B0A4D013CE4B2029400240F4B48
:10AF000001940095FFF792FD041E00D014E1290082
:10AF10007888FAF735FFDFE6A86CFF1F2444FF1F8F
:10AF2000AC69FF1FA069FF1FA66AFF1FDC65FF1F3A
:10AF30009C6BFF1F2244FF1FFFFF0000AE69FF1F35
:10AF4000162406ABE41821003889FCF753FD011ED6
:10AF500000D182E178882288AE4C45002C5BAE4D52
:10AF6000013CE4B202947C89AC4B01940095FFF75C
:10AF70005DFD041E00D0DFE029007888FAF70AFFA3
:10AF8000AAE60025A44B1D803B00FE331B78A24A95
:10AF900078880792AB4208D99E4B1288069306998F
:10AFA00043005B5A013B9A4203DB0799FAF7FCFE28
:10AFB00092E616246B00FB18059306ABE418059B7C
:10AFC00021001889FCF716FD011E03D1059B012401
:10AFD0001E8973E77888924B2288069C0993430068
:10AFE0001B5B904E013BDBB2029300230096019362
:10AFF000099BFFF71BFD041E02D0059B1E895DE720
:10B000007B88069A5B009B5A079A10883288121830
:10B01000934202DC1B1A013B33807F4C02303288A2
:10B020000999001900F01CFB2388328801359B1810
:10B030002380EDB2A8E70BAA3B7B7989388900927F
:10B040003A000D32FCF7EEFB00250590059B002B26
:10B0500004D10A24002D00D16EE060E0059B7888C1
:10B06000197AFCF7A9FB0100041E63D1694C6C4BF3
:10B07000788806940993069B4400E45A694B063C81
:10B08000E4B20BAE328807930294019100930599C4
:10B09000099BFFF7CBFC041E4CD1079B5E491B8824
:10B0A0001A1D002D30D14A80059B5B4C5A896319CB
:10B0B0001A716B1C9BB2E318120A1A71162306A8A8
:10B0C00032881B1879890598FCF708FDFF21AA1C16
:10B0D0002E1D03350B00059092B2B6B2ADB200281A
:10B0E00003D006ABDB8AD9B21B0AA218651911710D
:10B0F0002B714C4D301D2A884949201800F0B0FAB8
:10B100002B88F618B5B2A1E74988914207D17A8811
:10B1100006995200525AEB18053A9A42C4DC3E4C4A
:10B120002800618800F0B4F9207021007888FAF7CF
:10B1300045FED1E5002DF2D13E89BFE6162606ABCD
:10B14000F61831003889FCF755FC3D000400FF3546
:10B1500000282DD0037A9B060CD400227B893989E4
:10B16000788800923A000C32FFF7E8FB041E10D0FA
:10B170003E8915E03088FFF741FB00281AD083682C
:10B18000002B17D02100122278889847041EE4D0A3
:10B19000EEE7AB78002B02D17888FAF71FFE002685
:10B1A000AB78002B00D097E5002C00D194E585E624
:10B1B0000124DDE70E24DBE7162506ABED18290098
:10B1C0003889FCF717FC041E47D0037A9B0611D47C
:10B1D000154A7B881188994203D01448814207D1CF
:10B1E0001380134BF8261D780023D9B2A94221D32E
:10B1F0000924A1E72888FFF701FB00282FD08368E6
:10B20000002B2CD02100122278889847041EDFD012
:10B2100092E7C046DC65FF1FAC69FF1FAE69FF1FE8
:10B22000A66AFF1F9C6BFF1FA06CFF1FFFFF0000A3
:10B230009C6CFF1F31005943546801336018615AF8
:10B240000029D2D13C0008342100F82200F008FA8D
:10B2500021007888FAF7CAFD3EE501246CE70E2448
:10B260006AE71D4B1A887B889A4231D07888FAF7B2
:10B27000C7FD31E5F823059851684343CD18C95AF5
:10B2800000291FD03B7A012B0BD16C88AB887888C2
:10B29000AA1D0094FFF752FB041E02D000233B724C
:10B2A0002E88F8220021280000F0EAFA00232B80E3
:10B2B000059B0133DBB20593084B05991B78064AC1
:10B2C0008B42D7D801235B421380002CCED0F5E50A
:10B2D000002634000596EFE7A06CFF1F9C6CFF1F53
:10B2E00070B504000E001500FFF796FA031E08D192
:10B2F00031000548FFF790FA03001120002B02D01F
:10B300001C8000209D7070BDFFFF0000F8B50B4F42
:10B3100006003B780D001400FF2B0ED00A2000F031
:10B32000EFF8011E09D0B12303800023468003718A
:10B33000C5800481387800F003FAF8BD7945FF1F15
:10B34000F7B50F0008A90600088809A90B24098889
:10B35000002821D10234022B1ED1557813782D02FA
:10B360001D432B008B4301937334002B14D1FB68D6
:10B37000300019000093FFF74FFB019C85420BD072
:10B380002A0030000099FFF7ABFF041E04D12A0009
:10B3900030007989FFF7BAFF2000FEBDF0B50E78C6
:10B3A00085B003900AA805880120022E0DD14C68B3
:10B3B0002778647824023C43054FBC4205D10398AA
:10B3C000DBB201960095FFF7BBFF05B0F0BDC046AC
:10B3D0000229000010B504000C4800F061FB0C4885
:10B3E000A16B00F05DFB0B48E16B00F059FB0A48D4
:10B3F000216C00F055FB094B0948196800F050FB1F
:10B40000084B1B68002B00D09847FEE726BC0011B4
:10B410003CBC00114BBC00115ABC001104ED00E013
:10B4200069BC0011AC6CFF1F002307B501A8019394
:10B43000FFF7D0FF044A0548002110B5121A00F0AA
:10B440001FFAF8F7B9FAFEE7B06CFF1F7C45FF1F43
:10B4500001B40248844601BC604700BFF136FF1FBB
:10B4600001B40248844601BC604700BFDD520100C0
:10B4700001B40248844601BC604700BFC53F0000DC
:10B4800001B40248844601BC604700BF5D1700005C
:10B4900001B40248844601BC604700BF090E0000A9
:10B4A00001B40248844601BC604700BF7D18FF1FFD
:10B4B00001B40248844601BC604700BF0D52010040
:10B4C00001B40248844601BC604700BF851F0000EC
:10B4D00001B40248844601BC604700BF55490100E1
:10B4E00001B40248844601BC604700BFA134FF1F7D
:10B4F00001B40248844601BC604700BFA54F01006B
:10B5000001B40248844601BC604700BF1D4D0100E4
:10B5100001B40248844601BC604700BFE537FF1F05
:10B5200001B40248844601BC604700BF091B00000B
:10B5300001B40248844601BC604700BF291C0000DA
:10B5400001B40248844601BC604700BF25260000C4
:10B5500001B40248844601BC604700BFE139FF1FC7
:10B5600001B40248844601BC604700BF810E000060
:10B5700001B40248844601BC604700BF791800004E
:10B5800001B40248844601BC604700BF5522000058
:10B5900001B40248844601BC604700BF8D3AFF1FDA
:10B5A00001B40248844601BC604700BF5125000039
:10B5B00001B40248844601BC604700BFF94C010059
:10B5C00001B40248844601BC604700BFA94601009F
:10B5D00001B40248844601BC604700BF1D4B010016
:10B5E00001B40248844601BC604700BF691F0000E7
:10B5F00001B40248844601BC604700BF6571010088
:10B6000001B40248844601BC604700BF056A0000DF
:10B6100001B40248844601BC604700BF0933FF1FE4
:10B6200001B40248844601BC604700BF350E0000EB
:10B6300001B40248844601BC604700BF3555000094
:10B6400001B40248844601BC604700BF093BFF1FAC
:10B6500001B40248844601BC604700BFE9280000ED
:10B6600001B40248844601BC604700BFE94C0100B8
:10B6700001B40248844601BC604700BFC95C0100B8
:10B6800001B40248844601BC604700BFC5210000E8
:10B6900001B40248844601BC604700BFC132FF1FAD
:10B6A00001B40248844601BC604700BF8B520100D0
:10B6B00001B40248844601BC604700BF3D4B010015
:10B6C00001B40248844601BC604700BF5118FF1F07
:10B6D00001B40248844601BC604700BFC94A01006A
:10B6E00001B40248844601BC604700BFC92600007F
:10B6F00001B40248844601BC604700BFD94901003B
:10B7000001B40248844601BC604700BF75A900002F
:10B7100001B40248844601BC604700BF0124000018
:10B7200001B40248844601BC604700BFE117000035
:10B7300001B40248844601BC604700BF8D1200007E
:10B7400001B40248844601BC604700BF594F010064
:10B7500001B40248844601BC604700BF5952010051
:10B7600001B40248844601BC604700BF593CFF1F3A
:10B7700001B40248844601BC604700BF151BFF1F8F
:10B7800001B40248844601BC604700BF350E00008A
:10B7900001B40248844601BC604700BFD91B0000C9
:10B7A00001B40248844601BC604700BFB14E0000AE
:10B7B00001B40248844601BC604700BF85520100C5
:10B7C00001B40248844601BC604700BF9130FF1FAE
:10B7D00001B40248844601BC604700BFA139FF1F85
:10B7E00001B40248844601BC604700BFB70E0000A8
:10B7F00001B40248844601BC604700BFADAE000002
:10B8000001B40248844601BC604700BF5539FF1FA0
:10B8100001B40248844601BC604700BF090E000025
:10B8200001B40248844601BC604700BF4D1F0000C0
:10B8300001B40248844601BC604700BFE5480000EF
:10B8400001B40248844601BC604700BF311B0000C0
:10B8500001B40248844601BC604700BF6932FF1F43
:10B8600001B40248844601BC604700BFEDA500005A
:10B8700001B40248844601BC604700BF5147010043
:10B8800001B40248844601BC604700BF154D010069
:10B8900001B40248844601BC604700BF6DBC000093
:10B8A00001B40248844601BC604700BFD1A5000036
:10B8B00001B40248844601BC604700BFC51D0000BA
:10B8C00001B40248844601BC604700BF1147010033
:10B8D00001B40248844601BC604700BF055E000019
:10B8E00001B40248844601BC604700BFDD30FF1F41
:10B8F00001B40248844601BC604700BF3D18000007
:10B9000001B40248844601BC604700BF0134FF1FF8
:10B9100001B40248844601BC604700BF45500000A6
:10B9200001B40248844601BC604700BFC56D0100F8
:10B9300001B40248844601BC604700BF6939FF1F5B
:10B9400001B40248844601BC604700BF014C0100BD
:10B9500001B40248844601BC604700BF017F00007B
:10B9600001B40248844601BC604700BF9135FF1F07
:10B9700001B40248844601BC604700BFF54E010097
:10B9800001B40248844601BC604700BF313CFF1F40
:10B9900001B40248844601BC604700BF2124000076
:10B9A00001B40248844601BC604700BF0189000021
:10B9B00001B40248844601BC604700BFB54C010099
:10B9C00001B40248844601BC604700BF8132FF1FBA
:10B9D00001B40248844601BC604700BFCD4C010061
:10B9E00001B40248844601BC604700BF1537FF1F01
:10B9F00001B40248844601BC604700BF453CFF1FBC
:10BA000001B40248844601BC604700BF21460100E2
:10BA100001B40248844601BC604700BF9DA90000F4
:10BA200001B40248844601BC604700BF456B010079
:10BA300001B40248844601BC604700BFC9A90000A8
:10BA400001B40248844601BC604700BF4551010073
:10BA500001B40248844601BC604700BF295101007F
:10BA600001B40248844601BC604700BFED4A0100B2
:10BA700001B40248844601BC604700BFB3520100D4
:10BA800001B40248844601BC604700BF353BFF1F3C
:10BA900001B40248844601BC604700BF213AFF1F41
:10BAA00001B40248844601BC604700BFE53A01008A
:10BAB00001B40248844601BC604700BF4134FF1F07
:10BAC00001B40248844601BC604700BFF30E000089
:10BAD00001B40248844601BC604700BF434D0100E9
:10BAE00001B40248844601BC604700BF9938FF1F7B
:10BAF0000002010302020303040305020602070217
:10BB0000080209030A030B030C020D020E030F03C4
:10BB1000100311031303140315001600793D0011DF
:10BB2000AD3D0011000000000200000032BB00111A
:10BB3000192A0F180A000000F1590000FD24000026
:10BB400041460100317E0011459E0011997200119D
:10BB5000357C0011CD5100116DAC00117D4E0011EE
:10BB6000713F0011A14000110000000016160000F6
:10BB7000020000007CBB0011F4FFF3FFD2FC0000C8
:10BB8000854100110000000000000000547579613B
:10BB90000056302E370030303031006769746875D8
:10BBA000622E636F6D2F70767678005448303500C2
:10BBB00002000000C4BB0011292A282A272A262AAD
:10BBC000252A242A0A180000E2040000710200005D
:10BBD00078EC0000744000001027000060F00000C6
:10BBE00006640000204E000000000000000000007D
:10BBF0001F501D00023C020000011500070000005C
:10BC0000A3020000303132333435363738394142FF
:10BC100043444546005048592B36325858504C55ED
:10BC20005330353034005B48617264206661756C56
:10BC3000742068616E646C65725D0A004C5220204D
:10BC4000203D203078253038780A005043202020CD
:10BC50003D203078253038780A0050535220203D5E
:10BC6000203078253038780A0049435352203D204F
:10BC70003078253038780A00DD5500113156001132
:10BC8000000000000200000090BC00116F2A6E2A24
:10BC90001A18D880F060FFFFFFFFFFFFFFFFFFF3E0
:10BCA00003B59747D6F613F7D777E6F0A7F47400F5
:10BCB000000001A0000000006410B71DC8206E3B0A
:10BCC000AC30D9269041DC76F4516B6B5861B24DA3
:10BCD0003C7105502083B8ED44930FF0E8A3D6D60D
:10BCE0008CB361CBB0C2649BD4D2D38678E20AA075
:10BCF0001CF2BDBDFB349B5F800000800010000083
:10BD0000000000009B5E001125750011BF5E001150
:10BD10002D790011435F001103790011B95F001103
:10BD2000D97800110B600011A17A00117360001125
:10BD3000A17A0011A56000115B7A0011B95F0011B2
:10BD40009178001131600011397A00110000000073
:10BD50000000000017610011397A001179610011AB
:10BD60003D750011052A042A012A002A0229032808
:10BD70000128002801180018000000000000000041
:10BD80000000000000000087010102010201010221
:10BD90000102030304010301010101010303020184
:10BDA00003000D000E001000110013001401070124
:10BDB00008010A010B011C011D0204020502070211
:10BDC000080219021A021C021D03010302031700D4
:10BDD0000201000504000807000B0A001716001DE9
:10BDE0001C010201010504010E0D011110011413C3
:10BDF000011716011A19020201020B0A020E0D02A6
:10BE00001110021413021716030504030807030B8D
:10BE10000A030E0D0001020307090A0B0E0F101191
:10BE200012141718191A1B1F20212200B5A5001182
:10BE300071A60011000000000200000076BD001194
:10BE4000000000009DB3001100000000020000008F
:04BE500074BD0011AC
:020000041FFFDC
:1000000000000000D53E001138BB001134BB0011C8
:100010008862FF1F000000000000000000000000D8
:1000200000000000000000000000000000000000D0
:1000300000000000000000000000000000000000C0
:1000400000000000000000000000000000000000B0
:1000500000000000000000000000000000000000A0
:100060000000000000000000000000000000000090
:100070000000000000000000000000000000000080
:100080000000000000000000000000000000000070
:100090000000000000000000000000000000000060
:1000A0000000000000000000000000000000000050
:1000B0000000000000000000000000000000000040
:1000C0000000000000000000000000000000000030
:1000D0000000000000000000000000000000000020
:1000E0000000000000000000000000000000000010
:1000F0000000000000000000000000000000000000
:1001000000000000000000000000000000000000EF
:1001100000000000000000000000000000000000DF
:1001200000000000000000000000000000000000CF
:1001300000000000000000000000000000000000BF
:1001400000000000000000000000000000000000AF
:10015000000000000000000000000000000000009F
:10016000000000000000000000000000000000008F
:10017000000000000000000000000000000000007F
:10018000000000000000000000000000000000006F
:100190006534FF1F5533FF1FC166010000000000DA
:1001A000000000000000000000000000000000004F
:1001B000000000000000000000000000000000003F
:1001C000000000000000000000000000000000002F
:1001D000000000000000000000000000000000001F
:1001E000000000000000000000000000000000000F
:1001F00000000000000000000000000000000000FF
:1002000000000000000000000000000000000000EE
:1002100000000000000000000000000000000000DE
:1002200000000000000000000000000000000000CE
:1002300000000000000000000000000000000000BE
:1002400000000000000000000000000000000000AE
:10025000000000000000000000000000000000009E
:10026000000000000000000000000000000000008E
:10027000000000000000000000000000000000007E
:10028000000000000000000000000000000000006E
:10029000000000000000000000000000000000005E
:1002A000000000000000000000000000000000004E
:1002B000000000000000000000000000000000003E
:1002C000000000000000000000000000000000002E
:1002D000000000000000000000000000000000001E
:1002E000000000000000000000000000000000000E
:1002F00000000000000000000000000000000000FE
:1003000000000000000000000000000000000000ED
:1003100000000000000000000000000000000000DD
:1003200000000000000000000000000000000000CD
:1003300000000000000000000000000000000000BD
:1003400000000000000000000000000000000000AD
:10035000000000000000000000000000000000009D
:10036000000000000000000000000000000000008D
:1003700029B400110000000000000000000000008F
:10038000000000000000000000000000000000006D
:10039000000000000000000000000000000000005D
:1003A000000000000000000000000000951AFF1F80
:1003B000000000000000000000000000000000003D
:1003C000000000000000000000000000000000002D
:1003D000000000000000000000000000000000001D
:1003E000000000000000000000000000000000000D
:1003F00000000000000000000000000000000000FD
:08183800B070FF1F4118FF1FF3
:10184000024981F3088802F00BFC0000B070FF1F12
:1018500010B502F03DFA072804D0122808D002285B
:1018600008D010BD044A0420136B01331363F8E75A
:101870000220F6E71420F4E78466FF1FF8B507009E
:101880000C0026002500503630785135002804D150
:101890000300287058342370F8BD2978CA00481E08
:1018A0008141A3183800A25C5B68C9B2FFF7D0FF82
:1018B00000280DD12B78DA00A218013350602B706C
:1018C0003378044A013B3370136A01331362D8E75B
:1018D0000123DFE78466FF1F5C234343074910B5FC
:1018E000C9180B0058331B78012B05D1FFF7C6FF31
:1018F000034A936A0133936210BDC046B866FF1F66
:101900008466FF1F10B502F063FB064A0121130035
:1019100010CB4942D967044B136002F0D1FB200081
:1019200010BDC04600E100E01000100010B504003A
:1019300002F04EFB024B1C6002F0C2FB10BDC04621
:1019400000E100E010B5040002F042FB4021094A2A
:10195000200013688B43136002F0CAFB01F064FDA2
:101960000022054B01201A60044B04321A6002F079
:10197000AFFAFEE71CF00040C4F00040C0F00040A9
:10198000431E5A425341A022F0B5D2015B4213409C
:10199000154D164A40019B182A18127E8BB00191F2
:1019A000002A1BD01A000832D46F0022E6B206AF1C
:1019B000E4B294420EDC2818C369002B08D00199C8
:1019C00002AA117106AA049202AA167303A89847E4
:1019D0000BB0F0BD1978B9540132EAE71A7D1A78D4
:1019E00006AB01261A70E6E74469FF1F004000407D
:1019F000F0B5254B04004001C25C85B0002A2BD015
:101A00001A18117E002927D0917E002924D011793F
:101A1000022921D11689D788D168F51BADB22A1CBD
:101A2000102D00D9102292B2BE4217D118180123EE
:101A300003710023C269C38003819A4206D06846BD
:101A4000032103730171029301A890470820002C21
:101A500000D0192001F034FC05B0F0BD013C654216
:101A60006C41A0256442ED012C40084D1B186419FF
:101A7000074D0633013A92B2AA42EDD01888461CAF
:101A80001E80085C2070F5E74469FF1F004000409D
:101A9000FFFF00000F220E4B10B59868104002386F
:101AA0000A280BD802F0CEF80D0A0B0A0A110A0A0E
:101AB0000A0A060002210020FFF762FF10BD012183
:101AC000F9E70020FFF794FFF8E7DB6FF6E7C04681
:101AD000004000400F220E4B10B5986810400238AD
:101AE0000A280BD802F0AEF80E0A0B0A0A120A0AEC
:101AF0000A0A060002210120FFF742FF10BD012162
:101B00000800F9E70120FFF773FFF7E7DB6FF5E760
:101B10000090004013B5334C2378072B3DD8324B4F
:101B20001A78324B002A39D18022196852020A43AE
:101B30001A60252001F034FF20232D4A11680B4341
:101B4000802113606B460422C905086807331042E0
:101B500028D080210422C905C86810422ED08021D7
:101B60002020C905CA688243CA6014221A701A78F4
:101B7000002A2FD18021C905C86820320243CA60DB
:101B800014221A701A78002A28D11A4B1A7D22784A
:101B90005A601D221A705932DA6013BD1A6816494C
:101BA0000A40C5E7086802430A6014221A701A78CE
:101BB000002ACED01A78013AD2B2F7E7C8680243B9
:101BC000CA6014221A7019784A1ED2B21A700029FB
:101BD000F9D1C4E71A78013AD2B2C7E71A78013AC4
:101BE000D2B2CEE7B444FF1F7C45FF1F3CF000405B
:101BF000AC44FF1F00200040FFFFFEFF564B70B5B6
:101C00001B68012B03D1554A936D0133936502F094
:101C1000D7F9534B534A1860534B544C1A60012365
:101C2000534A1360534A13602378002B06D00622D0
:101C30005149524802F03CF900232370504A514B5D
:101C400010681B78C1B2002B0ED14F4CC0B2237864
:101C50005BB2002B4FDB237824785BB264B21B04A9
:101C600024021B191B1813600B1C50294ED950233A
:101C7000464A47491078DBB2FF2202284BD1086858
:101C8000444C454D267890432A78964254D9227880
:101C900024782E78023B5D10A31B6B435201D31AAC
:101CA00010335B111843086002F02AF8031F012B60
:101CB00045D83A4B1B78002B06D0394B1B78002BAC
:101CC00002D0002002F01CFAA122364B9200997833
:101CD000354B4A431B689B18832292009B181B7844
:101CE000033B012B03D8AF20400002F051FA012240
:101CF0002E4BDA8270BD237824785BB264B2FF3356
:101D0000FF341B0424021B190138ABE7CAB2022AB4
:101D1000AED20223ACE70868254C264D26789043C6
:101D20002A78964208D9227824782D78023B5B10D5
:101D3000641B63435201B2E72378DBB2B2E70228A7
:101D4000D5D11D4B1B78013B022B03D91B4B1B78B4
:101D5000022BCCD16C20C8E79809FF1FFC0FFF1F96
:101D6000BC65FF1FFF3F000014100340C065FF1F4C
:101D70000C10034000100340D50BFF1F7211FF1F12
:101D8000B40003408C09FF1F680AFF1F490AFF1FA8
:101D900094000340460AFF1F470AFF1FF908FF1F70
:101DA0002209FF1F300DFF1F3409FF1FBC0BFF1F4F
:101DB000440AFF1F450AFF1F1C09FF1F2309FF1FBD
:101DC00010B502F085F90022014B1A8010BDC04603
:101DD000B865FF1F10B502F083F8A121054A8900FC
:101DE0009478054A61431268044B5218528C1A8049
:101DF00010BDC046300DFF1F3409FF1FB865FF1F1F
:101E000010B50D4B0D4A9978A1239B004B431268E6
:101E1000D218531DD97F0A4B1B88994209D2441C02
:101E200007D0C82805D0D2695B1A5A43054B5343E3
:101E3000C01802F025F810BD300DFF1F3409FF1F38
:101E4000B865FF1F7102000070B5244D2B68002B90
:101E500028D002F02DF92B68D8402B680400002B05
:101E600027D001F085FF2B68D8401D4B1D4A99787B
:101E7000A1239B004B431268D118D25C91239B0095
:101E8000002A20D0CA580132CA50174B17491B6884
:101E90000868834214D3D23B181A012A1AD0144B73
:101EA000186070BD02F004F9124B196801F000FFD0
:101EB000D3E701F05DFF0F4B196801F0F9FED4E79D
:101EC0000D495B18E8E7CA500C4B1B68DB68E41847
:101ED000201AE4E7F530FF30E1E7C0461C08FF1F99
:101EE000300DFF1F3409FF1F9C09FF1FBC65FF1F3A
:101EF000A009FF1F1808FF1F2DFF3F00C465FF1F2B
:101F000070B504000D00282916D10300A433C2883F
:101F10001B889B1A0B4A9BB293420DD906006A3666
:101F200005223100653002F00BF9002804D13100A0
:101F3000200002F01DF870BD2900200001F078FF9C
:101F4000F9E7C046FE7F0000F8B50400012002F06A
:101F500017F801F0A5FE174A174910600968030039
:101F60001648174E01601748776805680020AF4291
:101F700001D27068281A144D091928601348C162EB
:101F8000A421446A49032143416211490978002987
:101F900005D010490978022902D10F3B1360F8BD22
:101FA000012901D1083BF9E7032901D1053BF5E7F8
:101FB000033BF3E7E408FF1F28F00040340AFF1F4B
:101FC00028100040180AFF1F1C0AFF1F00F00040E5
:101FD0001C09FF1F4A0AFF1F70B580241025E40565
:101FE000A3682B43A36002F0CBF8A368AB43A360C4
:101FF00070BD0000F7B5160080221C001023D2052A
:102000000191916805000B43936000225A4BD73031
:102010001A6001F055FE9D232A002F009B00EB580B
:10202000CA3201210092FC37002B01D00021009A16
:10203000386802F0BDF82900009BCB311A784F4B6D
:10204000D3351A604B780A781B0213438A7812043E
:102050001A43CB781B061343494A1BBA13604B79CA
:102060000A791B0213438A7912041A43CB7931008F
:102070001B061343434A1BBA13606B782A781B0272
:102080001343AA7812041A43EB781B0613433E4A03
:102090001BBA1360019A330213433C4A13603C4B52
:1020A00022001B1B9C4603293DDCB3089A00130049
:1020B0005142B21A032A46D1354AE018511A8278A1
:1020C0004078120400020243E05C043302430A60D9
:1020D0000022FF2B4BDDF0222E4B12011A600F2243
:1020E0002D4B1A602D4A1368002BFCD00023224A86
:1020F00027491360091B321D0B191B68043A180A83
:1021000023706070180C1B0EA070E3700434002A5A
:10211000F2DC802210213B68D20501333B609368DA
:102120008B439360F7BD6346D578981893782D0656
:102130001B042B43157804392B43557804322D02A8
:102140002B430360AFE7022A0AD1114AE05C511A1F
:10215000E2185278120202430A6004339BB2B7E7D6
:10216000012AB5D10A4A521AE15C1160F5E7084923
:1021700059180A600433ACE7000004403C000440F6
:102180003800044034000440300004400C00044097
:102190000001044004000440100004401400044006
:1021A000F7B5150080221C001023D205009191681C
:1021B00007000B4393600023654AD730136001F09A
:1021C0007FFD9D233E009B00F9583B00CA3632003C
:1021D000FC33002900D07FE0586801F0E9FF3900A6
:1021E00032785C4BCB311A604B780A781B02134370
:1021F0008A78AC4612041A43CB78281D1B06134379
:10220000554A1BBA13604B790A791B0213438A792A
:1022100012041A43CB791B061343504A1BBA1360AE
:102220004B7A0A7A1B0213438A7A12041A43CB7A36
:1022300021001B0613434A4A1BBA1360009A2B0263
:102240001343484A13602200474B1B1B0093009B1B
:10225000CE785B1801938B7836061B0433430E78D7
:10226000043833434E78043136023343019E3360E1
:102270000328ECDC0321A808431C9B0029408000B4
:1022800003292BD13849E5185E18A9786D78E35CED
:1022900009042D022943194331600300083300214A
:1022A000FF2B2DDD314B324919600F21314B196065
:1022B000012327490B60304B19680029FCD0062107
:1022C0001B680B40042B20D080220020D20593688D
:1022D0000A318B439360FEBD01217DE7022908D1BD
:1022E00021495D18E1184978E35C09021943296026
:1022F000D3E70129D3D11C495918E35C0B60CCE723
:102300001948181801600433CAE7002310490B600C
:102310006346002B0CDC3B00FC335A681021013271
:102320005A608022D205936801208B439360D2E7E4
:10233000009B9B181B68190A13705170190C1B0E17
:10234000D37004235B4291709C440432E0E7C046A2
:10235000000004403C0004403800044034000440C5
:10236000300004400C00044000010440040004401C
:10237000080F0000100004401400044070B5061E51
:1023800019D00222614B9B799343012B13D1604BEF
:102390001A78FF2A0FD15A78FF2A0CD19A78FF2A8F
:1023A00009D1DA78FF2A06D11A79FF2A03D15B799D
:1023B000FF2B00D1A7E0574B0C201A78012A08D038
:1023C0000022554D1A702B781A00093A042A01D8B8
:1023D000212070BD5A1F012AFAD94C4CA07B042839
:1023E00000D990E0A279032A00D98CE0821E012A4C
:1023F00003D862881F2A00D885E0002E61D0012E04
:1024000000D080E0A288012AE2D0002B0AD1013856
:10241000032803D801F016FC151D19151F202E7076
:1024200001F036FE2B785A1E032A16D800253B4BA6
:102430001D602823237501F0B3FDA8422ED0A5808E
:10244000C6E7022320202B70EAE7042322202B700A
:10245000E6E7032321202B70E2E7073B012BB7D8E7
:102460002F4B1B68DB6A9B06B2D52E4B1A78002ACD
:10247000AED1A27B911E012901D9002AA8D1022246
:1024800080211A702823284D89012878237501F0AE
:1024900017FD80212878890101F04AFE0123A380DD
:1024A000224B1B78002B0AD0FA228021204B92006D
:1024B0001B8809025A431C4B187801F0A9FC002024
:1024C00087E701F085FD2B78A680073B012B06D915
:1024D00018482E7001F074FC1E2001F0D9FD114B3C
:1024E000114C1A78002A06D0802100222078890118
:1024F0001A7001F0E5FC01F0E3FD8021207809026B
:1025000001F0DEFCDBE7122063E7C046A60BFF1FED
:102510006B09FF1F1A09FF1F1C09FF1F4809FF1F36
:10252000C465FF1F2309FF1F1B09FF1F2109FF1F90
:102530002C09FF1F0010004010B5002901D001F048
:10254000A7FC10BDF7B5604B01919978A1239B00C2
:102550004B435E4A060014681022E418D6235B0041
:10256000E0583623FF33E35C00279343222B41D10D
:10257000574B0F3A1A600760012501F0D1FB019B10
:102580001880E8235B00E35C002B01D0B34258DDE8
:102590000023504FFB70AD33FF33E3581A68002A15
:1025A00003D09B88DB439B071DD03823FF33E35CBC
:1025B000002B18D09B235B00E35C002B13D1D1339D
:1025C000FF33E35CB3420EDAA4235B00E15AE01868
:1025D000090A023101F054FB23000122FE33013EBF
:1025E00001351A87FA70E8235B00E35C002B2AD0E0
:1025F000A8B2FEBD03683D00002BBED08188043028
:10260000090A023101F03CFBD6235B00E3581F604E
:10261000B2E72300B133BA00FF33985801378188FD
:102620000430090A023101F02BFBE8235B00E35C74
:10263000BB42EEDCE822F61AED1800235200A35448
:10264000A6E70027F1E7200001F0CAFC00281FD010
:10265000002E1DDD7319882647190193B60020004E
:1026600001F04EFC5A308000201840680135818806
:102670000430090A023101F003FB200001F030FDB3
:10268000A3590133A351BD4202D0019B9D42E6D123
:10269000114BE35C002BABD095239B00E35C002B3C
:1026A000A6D00E4BE15A0029A2D00D4AA35C994254
:1026B00002D90133A3549BE700231A212000A3541D
:1026C00001F0BEFC94E7C046300DFF1F3409FF1F28
:1026D00000140340E010FF1F5A02000072020000C5
:1026E0005E020000F8B51D4B1D4F1A78002A10D16C
:1026F000BA7B002A02D101321A7003E0032AFAD011
:10270000022AF8D001F04CFC00220120154B1A706F
:10271000F8BD154B154D1C68154B9E7801232B7089
:102720002878C0B200F0DEFCBB7B002B0BD101F09F
:102730000FFDA1239B007343E41883239B00E4183F
:1027400023782B70E4E7032B02D101F0A1FAF0E724
:102750000020022BDCD101F0FBFBEAE71C09FF1F84
:10276000A60BFF1F2309FF1F3409FF1F490AFF1F84
:10277000300DFF1FF0B587B00EAD2F780FAD2D785F
:102780000593AC46634614000E4D0CAA12782E78C1
:1027900003930D9B009201932200059B029701F089
:1027A000D7FA2E70012C01D0042C08D180220649C2
:1027B0008B889343054A1278D20113438B8007B06C
:1027C000F0BDC0461C09FF1F6C11FF1F7809FF1FD9
:1027D0000B001B3B70B504003020E02B0DD813001C
:1027E000E025493BFF3B9BB2ED00AB4205D8034BD4
:1027F000200019825A8201F08BFC70BD8410FF1FEB
:1028000010B501F0DDFB054B00205B68052B04D9FA
:10281000034A5268D20200D4980810BD001000404C
:10282000FCE100E070B501F0D3FB0D4B1B68FC33FD
:10283000DC691D6AFFF7E4FF6419844204D2094B86
:1028400001241B68002B07D004220024064B1A70B9
:10285000064A93690133936101F032FC200070BD98
:10286000C465FF1F9809FF1F2309FF1FFC0FFF1FEF
:1028700070B50C4D2B68FC335C6A01F0A9FBFFF7C7
:10288000BFFF2B680025FC339B6AE318834204D208
:10289000054B1B68AB4200D1051B01F011FC280061
:1028A00070BDC046C465FF1F9809FF1FD722044BA7
:1028B00092009B5810B5002B00D0984710BDC04621
:1028C0000000FF1FF0B587B001F046F9FFF7EEFFFB
:1028D000CA4BCB4C04931B78022B45D1C94B1B68C8
:1028E000186A01F04DFBC84BC84A1A60C84BC94A68
:1028F0001A60A022C84B52001A60049B187801F09D
:1029000067FAC649C64801F033FCC649C64801F01B
:102910002FFC1022C54BFF201A60802252031A6040
:10292000802292031A60802212041A6001F0E8FBF0
:10293000012001F015FCFA20400001F001FA5820B6
:1029400001F026FCBA4801F0ABFA012001F070FB5F
:10295000072001F0EDFA2268B64B1A4084235B0091
:102960001343236007B0F0BD01F09AFBB24E029012
:10297000322001F005FB33681B0629D43C2001F00E
:10298000FFFA0F2001F0FCFA9C4B1B78012B00D1C1
:102990001EE180223368A94D134200D0A7E02B68C6
:1029A000032013432B6001F0EBFA01F079FB029B4B
:1029B0000299C31A5A1E814200D81A00A04B1A600D
:1029C000904B19681E2353439E4A9B18CB618AE79C
:1029D00001F066FB80239C4ADB02116803900B43E5
:1029E00013602268934B994F1A40282313432360A6
:1029F000032001F0C5FA03203D6801F0C1FA3B68ED
:102A00000320DB03DB0B009301F0BAFA3B68ED0314
:102A1000DB03ED0BDB0B8E4A0193AB18C22B30D8D6
:102A2000009B9B18C22B2CD8019B9B18C22B28D82B
:102A3000009B2A009D4200D21A00009B9D4200D9B3
:102A40001D00019B934200D21300019A954200D9C8
:102A500015005B1B122B14D80C22336814209343EF
:102A6000336033687B4A1340336001F089FA0821F0
:102A70003B682268DB038A432260774ADB0B1360E2
:102A80007FE7032001F07CFA3B68DB03DB0B059357
:102A900001F006FB039B0399C21A531E814200D822
:102AA00013006E4A93421BD9FF23356869492D0AEA
:102AB0001D4032686B1C1B060A401B0C134333601D
:102AC0000C23326800209A43083B1343336001F023
:102AD0001FFA6348634BA840984206DCFEF732FFBA
:102AE000019B009D0093059B95E75F48F6E7002357
:102AF0005E4F554A3B6080231168DB020B43136035
:102B000080222B68032013432B6001F039FA3B68C5
:102B1000052601333B6080232A685B0213432B6048
:102B20002268444B03201A40514B1343236001F0A9
:102B300027FA0821454B1A682368D2038B43236088
:102B4000454B023900931B68D20B4B439A420CD879
:102B50009B1A3B2B0BD8236846490B4023602B68FC
:102B60000B402B60444B1A601FE7D31AF1E7013E7C
:102B7000F6B2002ED4D123683E4A134023602B685E
:102B800013402B603B68042B07D9BFF34F8F3B4B9F
:102B90003B4ADA60BFF34F8FFEE780222B680320A9
:102BA00093432B6001F0ECF92268224B03201A407A
:102BB00028231343236001F0E3F9244B009A1B6898
:102BC000DB03DB0B1360082223689343236097E742
:102BD00007222C4D2B681340012B02D1002001F05D
:102BE000F7F8AB68284A02201340AB6001F0C8F93F
:102BF0008023AA685B001343AB60D6E64A0AFF1F36
:102C00005CF00040C465FF1F000003400180063DEA
:102C1000BC00034034080000A4000340710200001F
:102C200014100040FFFF3F002810004000E100E0CA
:102C30003075000000FEFEFFC4F0004044F000408C
:102C4000AC65FF1F7206000040F0004064F00040D9
:102C500091FCFFFFFF00FFFFB465FF1FE30C0000C6
:102C6000E88000005F361E0060361E001844FF1F1B
:102C700028000100FFFFFEFFB065FF1F00ED00E030
:102C80000400FA053CF00040FFFEFFFF694E336888
:102C900088331B6883F3088801F0EAF800F0C4FB6E
:102CA000654B664A1B68934207D0002001F030F95B
:102CB0000221634A13688B431360FFF703FE614BE5
:102CC000614C1878C0B201F08BF80023A360023386
:102CD000A3605E4B0120236001F052F90323A3603F
:102CE00001F0DEF9040001F06BF9050001F0D8F9FC
:102CF000574B186001F034F8564B1968621A531E8E
:102D0000A14200D213008022D203934201D39B023E
:102D10009B0A3268D16AC90700D478E04E491C0C7E
:102D200009689BB24C4359432402090A64180327DB
:102D30004A49FC3293680A6849489B1A494A4A4EF4
:102D400012684A499B18414A34609A183B400193E3
:102D5000036892089C46019B0A6063440360042B4D
:102D600003D901323B400A6003600B684049E41814
:102D7000200000F09DFF3F4F3D493B68C3183B607A
:102D80002000019301F0ECF83B4C2068081838490A
:102D90002060884205D9019B01333B6001F0E0F8D7
:102DA000216001F05DF8354B1B78002B0ED001F04F
:102DB00007F93168324B4A1B1B6812189A4233D20A
:102DC000591A4919091A2F4801F0D2F92E4C237AC1
:102DD000002B0FD001F0F4F83168E3684A1B121899
:102DE000934224D9591A4919091A284801F0C0F9FF
:102DF00000232372264B83F3088800F079FF02201A
:102E000001F046F9002001F083F800F0B9FFDC0181
:102E100099000234641A5900641A09214B43803323
:102E2000CB40A408E41882E7FA218900CBE71949CE
:102E3000DBE7C046C465FF1F0C0AFF1FB641210334
:102E400010000040490AFF1F14100040C409000090
:102E5000100AFF1F340AFF1F380AFF1F200AFF1F36
:102E6000280AFF1F1C0AFF1FA865FF1F240AFF1F57
:102E7000710200006008FF1F2C0AFF1F1C09FF1FC2
:102E8000E408FF1F00100040740BFF1F3C100040BF
:102E900000000020DC050000A022054B92009B589A
:102EA00010B5002B01D0984710BD00F0D1FFFBE713
:102EB0000000FF1FA122054B92009B5810B5002B6C
:102EC00001D0984710BD00F0C3FFFBE70000FF1FD3
:102ED000A222054B92009B5810B5002B01D09847B9
:102EE00010BD00F0B5FFFBE70000FF1FA322054B5C
:102EF00092009B5810B5002B01D0984710BD00F0F0
:102F0000A7FFFBE70000FF1FA422054B92009B5880
:102F100010B5002B01D0984710BD00F099FFFBE7DA
:102F20000000FF1F70B501F04BF8514B18600420F2
:102F300001F0AEF801F09CF80400C30702D400F0E1
:102F40002FFF70BD00224B4B1A604B4B1878013895
:102F500004282CD800F076FE03231B1F2700200036
:102F600001F056F80128ECD0444C2378042B71D1A1
:102F700001F016F9002806D000F0CAFE582001F032
:102F800007F902232370032001F082F8D9E720001B
:102F900000F00EFFE6E7200000F0C2FFE2E72000AD
:102FA00000F03EFFDEE7200001F002F8DAE700F073
:102FB000A7FE0500012808D1314B1B78053B012BEA
:102FC00003D82000FFF768FFCEE72C4B1B78022BBD
:102FD00001D0052B20D1022D28D12A4B9B7BAB435E
:102FE0001CD12000FFF766FF254B18780128BBD1C4
:102FF0006405B9D4234925224B7B034205D1233AEA
:1030000013405A42534126331A000B7D9342ABD9E9
:10301000322000F0F5FEA7E7022D07D1184B1B78F0
:10302000052B11D12000FFF753FFDDE7012D0BD158
:10303000012B03D12000FFF759FF95E7062B03D1A1
:103040002000FFF761FF8FE7200000F001FF022D55
:103050008AD1C9E7032B04D10B4B987C00F070FF99
:1030600091E7072B8FD1094B987B00F0F1FF8AE79E
:103070009C09FF1F9809FF1F9009FF1F2309FF1FCD
:103080001C09FF1FA60BFF1FBC0BFF1FD40BFF1F4C
:10309000FA210A4B0A4A49001A640A4A5A500A4A53
:1030A00004395A50094A08319A64094A5A50094A5F
:1030B0005C315A50084ADA667047C0460000FF1F6C
:1030C0007527FF1F7128FF1F2528FF1F7D23FF1F66
:1030D000E526FF1F011EFF1FD51DFF1F10B500F0C5
:1030E00099FD10BD8023F7B59C46264B264F0193D2
:1030F0002649274A274D284C284B02281AD16046DA
:1031000038600868264E3040802636033043086019
:1031100001990978002909D11660224A2A60224AB9
:103120002260E02219689143A03A1BE08021C90285
:103130001160F2E766463E600F68194E3E408027F8
:10314000FF023E430E600199097800290DD11760F6
:1031500001280ED1154A2A60154A2260E02219681A
:103160009143C03A0A431A60F7BD80218902116079
:10317000EEE7E0210F4A02432A600F4A22601A68F4
:103180008A43F0E74B0AFF1FE0000340D8000340EA
:103190009000034000000340500003404000034003
:1031A000FFFFE3FF0280063D804508220180063DC7
:1031B000806608220080069880550822F8B51E4BCC
:1031C00080261A68002014003440324232D11A6836
:1031D0001A4F32431A6001223B68063093433B602A
:1031E00000F0CEFE0122164D2B681E432E603B6878
:1031F0000A2613433B608027BF00124B1B683B42EB
:1032000011D1013EF6B2FF2E09D17E220E4B1C6871
:103210002B68E40B1440934323432B6005E0082004
:1032200000F0AEFEE9E7002EEFD180222B686008A7
:1032300093432B60F8BDC046C4F000405CF00040F2
:1032400018F0004068F0004060F0004010B500F059
:1032500047FD01215820034A00F09AFDFFF7AEFF19
:1032600010BDC046600AFF1F10B578220021034838
:1032700000F08EFE00F0D4FE002010BDCC68FF1FD1
:1032800070B5040000F0A4FE00230C200B4A0100DE
:1032900059438D18515C00290DD0A14208D101235A
:1032A00000246B7000F044FD00F00AFF200070BDA8
:1032B00001330A2BEBD11224F6E7C046CC68FF1F7E
:1032C00070B5040000F084FE002319001D000D4AB3
:1032D0001078002806D0A0420CD1557001310C3274
:1032E0000A29F5D1002B0AD100F09AFE00F0E8FE81
:1032F000002070BD5078461EB0411B18EEE700F06C
:1033000017FDF3E7CC68FF1FF7B504000C2000237E
:1033100084460E4D019267465F43E85D7E19A042E8
:1033200012D000280BD10A4B9C4662461B7808330A
:103330001370019B70707C557160B360FEBD0133EA
:103340000A2BE8D10320F9E70720F7E7CC68FF1F35
:10335000C868FF1F8021204BC9051B6870B58B60B2
:103360001E4BC1241A680123FF2013434B611C4BE1
:10337000A4001A681B4B00251A601B4B1A681B4BD4
:103380001A601B4B1A5982431A51C52292009C584D
:103390008443BF38204398509C58164804408020EE
:1033A000C001204398509858134C0002000A014372
:1033B0009950124B1B78DB08AB4201DC002070BD3A
:1033C0002378002B06D0A368002B00D09847013546
:1033D0000C34EEE71220F2E7B044FF1FAC44FF1FAD
:1033E000B0F00040C468FF1FB4F00040C068FF1F89
:1033F00000E100E0FF00FFFFCC68FF1FC868FF1F6F
:10340000030010B51F2809D8072200201340072405
:1034100004490A78A24313430B7010BD0023062011
:10342000F5E7C046C868FF1F034A04491368002037
:103430000B4013607047C0461CF00040FFFFC1FF07
:10344000054B06491B780A6805485B0702401B0BC1
:10345000134300200B607047C868FF1F1CF000403A
:10346000FFFFC1FF70B50C25FFF7EAFF0A4B1C7880
:103470000A4BE4086543ED18002C01D1200070BD13
:103480002B78002B06D06B68002B00D09847013CAE
:103490000C3DF1E71220F2E7C868FF1FC068FF1F6C
:1034A00007B50422074801A900F034F9019B013354
:1034B00005D18023044ADB0411680B43136000200C
:1034C0000EBDC0461C18001114F00040F0B50500F8
:1034D0002026184B87B00493049B002B03D11124A2
:1034E000200007B0F0BD002102220B0001910091E5
:1034F000052000F015FE02230F490A681A42FCD18C
:103500000596059C631E0593002CFAD10B4A13689F
:10351000002BFCDA0F276F440121380000F0E8FC93
:103520003B782B42DCD0052000F02AFD049B013BB8
:103530000493D1E7FFFFFF0790C8004000C8004098
:1035400007B500F045FD80220821D205936A01915C
:10355000002B01D10739916202210C4A11600199B7
:10356000481E01900029FAD1033111600531019103
:103570000199481E01900029FAD11160002B02D157
:103580008022D205936200F09BFD07BD00C0004081
:10359000F0B52D4C89B02378002B4FD1FEF7B2F94E
:1035A00002232A4F03903A681A42FCD12023069343
:1035B000069B5A1E0692002BFAD1254E3368002B2B
:1035C000FCDA0120FFF782FF011E02D0112009B0B2
:1035D000F0BD030003220190009005AD9F2000F094
:1035E0009FFD0321280000F083FC02233A681A4261
:1035F000FCD120230793079B5A1E0792002BFAD178
:103600003368002BFCDA0120FFF760FF0028DDD1D2
:103610000398FEF78BF9AA786B7811041B020B4311
:1036200029780B4363601300113B0A49052B07D827
:1036300001239340A3600B60012323700020C6E7A1
:1036400080231B03F6E7C0469844FF1F90C8004044
:1036500000C800409808FF1F1E4B30B55A68187804
:103660001D4B85B0D31859424B41012100930023D3
:1036700000F0C6FC194B1A4A02259A6300221A650B
:1036800010325A658022C4219D65164B1648D2021D
:10369000DA6789004258154B80241A4080231B04A6
:1036A00013434350642341200393E40500F078F969
:1036B000402000F075F96562039D6B1E0393002D99
:1036C000FAD103236362FFF73BFFA562FFF760FFB8
:1036D00005B030BDA444FF1F95FFFEF700C80040B1
:1036E000050001FF04E100E000E100E0FFFF00FF52
:1036F00010B5064B18705960FFF7AEFF002113207C
:10370000034AFFF701FE002010BDC046A444FF1F7E
:103710005936FF1FF0B5040085B003920291FEF701
:10372000F1F8882263035B0B52051A438023DB0503
:103730009D6A8023274F0092BA68002601901B03E0
:103740009A420CD9F82326001B041E401C4206D0C6
:103750008022214B52025E6219680A431A60002DD2
:103760000BD100F035FC02221C4B1A608023DB05D4
:103770005A62013A9A6200F0A3FC0023039A934232
:1037800020D1002D0AD100F023FC144B03221D6030
:103790008023DB055A629D6200F092FC8023BA68A8
:1037A0001B039A4208D9002E06D000220A4B0C496E
:1037B0005A621A680A401A600198FEF7B7F80020AA
:1037C00005B0F0BD009A0299D2181278CA5401339C
:1037D000D4E7C0469844FF1F00C8004000C0004026
:1037E000FFFFFEFFF0B587B0029103920400FEF7E1
:1037F00089F8019000F0ECFB802302250122234E82
:10380000DB0535605D629A6200F05AFC204F3B6830
:103810002B42FCD120230493049B5A1E0492002BBC
:10382000FAD11C4D2B68002BFCDA0120FFF74EFE6D
:10383000002802D0112007B0F0BD2000039A0299A1
:1038400000F0D6FA022304003A681A42FCD1202381
:103850000593059B5A1E0592002BFAD12B68002B6D
:10386000FCDA0120FFF732FE051EE3D100F0B0FBC9
:1038700080230322DB0535605A629D6200F020FC44
:103880000198FEF753F8E0B2D5E7C04600C000400B
:1038900090C8004000C80040F0B5802687B0040002
:1038A000FEF730F8F605B36A02250393029000F0A4
:1038B0008FFB0123244F3D607562B36200F000FC72
:1038C000224E33682B42FCD120230493049B5A1EC2
:1038D0000492002BFAD11E4D2B68002BFCDA01203C
:1038E000FFF7F4FD002802D0112007B0F0BD200042
:1038F00000F0BEF90223019032681A42FCD1202365
:103900000593059B5A1E0592002BFAD12B68002BBC
:10391000FCDA0320FFF7DAFD041EE5D100F058FBC6
:1039200080230322DB053C605A629C6200F0C8FBE6
:10393000039B002B01D1FFF703FE0298FDF7F6FF72
:103940006B461879D1E7C04600C0004090C80040DF
:1039500000C8004007B5000201910422000A01A935
:10396000FFF740FF0EBD000073B5050005240B4AAC
:10397000A3005B429B1819686B46DE1D300000F007
:1039800037FB022804D133782B55013CEFD276BDAA
:10399000052CFCD00128FAD10230F8E714090011F7
:1039A0001F2807D8012380228340D20591680B434A
:1039B000936070473F2808D8012380222038834035
:1039C000D20551690B435361F3E75F28F1D8012316
:1039D000802240388340D205116A0B431362E8E726
:1039E0001F2807D8012280218240C9058B68934394
:1039F0008B6070473F2808D8012280212038824000
:103A0000C9054B6993434B61F3E75F28F1D8012265
:103A1000802140388240C9050B6A93430B62E8E776
:103A20001F2810D880230200DB05153A1968012AE7
:103A300006D820229143196019680A431A6070471A
:103A400001228240F6E73F2811D880230200DB05DF
:103A5000353AD968032A06D810229143D960D9682B
:103A60000A43DA60EBE7012220388240F5E75F285D
:103A7000E5D842238022181A413B8340D205516A7F
:103A800099435162516A0B435362D8E710B5040061
:103A9000012813D1A022184992050B685B015B092C
:103AA00013430B60154B164A19681140154A0A4317
:103AB0001A60402219680A431A6010BD0028FCD120
:103AC00001000A2000F0DCFA21000B2000F0D8FAF7
:103AD000C0220A4B920019680A4340211A601A68F2
:103AE0008A431A60B022044912060B685B015B0925
:103AF00013430B60E1E7C04614F000401CF00040A7
:103B00007F00FEFF80FD010072B6074A1368013393
:103B100013600422054B1A600023054A13608022BB
:103B2000D2055360FEE7C0467808FF1FC0F0004092
:103B3000C4F00040044B054A1A60054B1A6000228D
:103B4000044B1A607047C046140AFF1F841E000011
:103B5000380AFF1FC4F000400023034A1360034AE1
:103B60001360034A1360704754F0004040F1004076
:103B700044F10040002310B5184C8AB00093019323
:103B80002378012B27D06946012000F059F900283D
:103B900017D1009B12490293019B06AA0393114B74
:103BA00002A81B680493104B1B68059300F0E8FA09
:103BB00010220E4906A800F0C3FA002804D1FF2302
:103BC000237000200AB010BD0123094A074902A84A
:103BD000237000F0D5FA0120F4E7C046C865FF1F46
:103BE00010290011082900110C29001120290011A9
:103BF000CC65FF1F13B501246946012000F020F9B0
:103C0000034B00940193FFF7B5FF200016BDC0469B
:103C1000BB0B000010B5FFF79FFFFFF7EBFF00287D
:103C200002D0024B984710BDFEE7C046E1A200005B
:103C300002B4714649084900095649008E4402BC45
:103C40007047C04602B4714649084900095C490002
:103C50008E4402BC7047C04603B471464908400018
:103C60004900095A49008E4403BC70470000000017
:103C700001B40248844601BC604700BFA96F01003F
:103C800001B40248844601BC604700BFC115010071
:103C900001B40248844601BC604700BF75F80000CB
:103CA00001B40248844601BC604700BFBD5C01000E
:103CB00001B40248844601BC604700BF090E000001
:103CC00001B40248844601BC604700BF894400003B
:103CD00001B40248844601BC604700BFE9270000E8
:103CE00001B40248844601BC604700BFED68010092
:103CF00001B40248844601BC604700BF79970000C8
:103D000001B40248844601BC604700BFDD0C0100DD
:103D100001B40248844601BC604700BF6DF6000054
:103D200001B40248844601BC604700BFCD0C0100CD
:103D300001B40248844601BC604700BF21A90000CD
:103D400001B40248844601BC604700BF85120100EF
:103D500001B40248844601BC604700BF9D6A000070
:103D600001B40248844601BC604700BFC16601003F
:103D700001B40248844601BC604700BF6D0B0100DE
:103D800001B40248844601BC604700BF855201006F
:103D900001B40248844601BC604700BF01670100CE
:103DA00001B40248844601BC604700BFDD0A01003F
:103DB00001B40248844601BC604700BF09340100D9
:103DC00001B40248844601BC604700BFC1A50000A1
:103DD00001B40248844601BC604700BFEDA5000065
:103DE00001B40248844601BC604700BF8914010049
:103DF00001B40248844601BC604700BF95730100CE
:103E000001B40248844601BC604700BF613701002D
:103E100001B40248844601BC604700BF8B520100D8
:103E200001B40248844601BC604700BFF53501007B
:103E300001B40248844601BC604700BF51B800008D
:103E400001B40248844601BC604700BFE1AC0000F9
:103E500001B40248844601BC604700BFE917010075
:103E600001B40248844601BC604700BFD54401004C
:103E700001B40248844601BC604700BFC9A90000E4
:103E800001B40248844601BC604700BF8937010085
:103E900001B40248844601BC604700BFE9D4000079
:103EA00001B40248844601BC604700BF8D11010087
:103EB00001B40248844601BC604700BFE94C0100E0
:103EC00001B40248844601BC604700BFB352010000
:103ED00001B40248844601BC604700BFA1AF0000A6
:103EE00001B40248844601BC604700BFF9ED000000
:103EF00001B40248844601BC604700BF3D71010027
:103F000001B40248844601BC604700BFD9B000003C
:103F100001B40248844601BC604700BF016C010047
:103F200001B40248844601BC604700BF053401006B
:103F300001B40248844601BC604700BFF90D01008E
:103F400001B40248844601BC604700BF4DF900003F
:103F500001B40248844601BC604700BF19FA000062
:103F600001B40248844601BC604700BF090E00004E
:103F700001B40248844601BC604700BF85C100000F
:103F800001B40248844601BC604700BF01890000BB
:103F900001B40248844601BC604700BFB70E000070
:103FA00001B40248844601BC604700BFA9D80000A4
:103FB00001B40248844601BC604700BFF9350100E6
:103FC00001B40248844601BC604700BFC95C0100DF
:103FD00001B40248844601BC604700BF75A90000D7
:103FE00001B40248844601BC604700BF71B00000C4
:103FF00001B40248844601BC604700BF91380011FB
:1040000001B40248844601BC604700BFC56D010091
:1040100001B40248844601BC604700BF013401007E
:1040200001B40248844601BC604700BFADAE000049
:1040300001B40248844601BC604700BFE51201009C
:1040400001B40248844601BC604700BF53B9000078
:1040500001B40248844601BC604700BFC1F70000BC
:1040600001B40248844601BC604700BF35B400116A
:1040700001B40248844601BC604700BFBD0B01008B
:1040800001B40248844601BC604700BF25A000116E
:1040900001B40248844601BC604700BF1907010013
:1040A00001B40248844601BC604700BF156B0100A3
:1040B00001B40248844601BC604700BFE90B01001F
:1040C00001B40248844601BC604700BF9DA90000BE
:1040D00001B40248844601BC604700BF8D820000E5
:1040E00001B40248844601BC604700BF5976010014
:1040F00001B40248844601BC604700BFF9A6000035
:1041000001B40248844601BC604700BFED6B01006A
:1041100001B40248844601BC604700BF116E000034
:1041200001B40248844601BC604700BF496D0100EC
:1041300001B40248844601BC604700BF0D52010033
:1041400001B40248844601BC604700BFCD4C010069
:1041500001B40248844601BC604700BFE9F6000094
:1041600001B40248844601BC604700BF69110100E8
:1041700001B40248844601BC604700BF2D6C0100B9
:1041800001B40248844601BC604700BFDD3F000027
:1041900001B40248844601BC604700BF79120100A7
:1041A00001B40248844601BC604700BF01D700004B
:1041B00001B40248844601BC604700BF21440000AE
:1041C0000200000072BD00110100000028BB0011B8
:1041D000020000006EBD0011010000000042FF1F40
:1041E0000200000030BB0011010000000863FF1F47
:1041F000020000006CBD0011030000007C62FF1F84
:10420000120000000200000072BD00110100000059
:1042100070BB0011020000006EBD00110100000023
:104220006DBB0011020000007ABB0011030000000A
:10423000B762FF1F020000006CBD00110300000008
:10424000CC62FF1F020000006EBD001101000000E3
:104250006CBB00110200000078BB001103000000DD
:104260008D62FF1F020000006CBD00110300000002
:10427000AE62FF1F0200000072BD001101000000CD
:10428000B0BB0011020000006EBD00110100000073
:104290004943FF1F02000000C2BB001101000000E3
:1042A000ABBB0011020000006EBD00110100000058
:1042B0004843FF1F02000000C0BB001101000000C6
:1042C000D462FF1F020000006EBD0011010000005B
:1042D0004743FF1F02000000BEBB001101000000A9
:1042E0009BBB0011020000006EBD00110100000028
:1042F0004643FF1F02000000BCBB0011010000008C
:1043000096BB0011020000006EBD0011010000000C
:104310004543FF1F02000000BABB0011010000006E
:1043200091BB0011020000006EBD001101000000F1
:104330004443FF1F02000000B8BB00110100000051
:104340008CBB00110202020202020000AD4A001101
:10435000AB4A001104BC0011900118001800FFFFC7
:104360000701020304050602010600000000000028
:10437000000000000000000000000000000000003D
:1043800000000000000003000200000072BD0011E8
:104390000100000084BC0011020000006EBD00118D
:1043A00001000000F843FF1F020000008EBC001156
:1043B000010000000263FF1F020000006CBD00113D
:1043C000030000007065FF1F020000006EBD0011B9
:1043D00001000000F843FF1F020000008CBC001128
:1043E000010000000463FF1F020000006CBD00110B
:1043F000030000006865FF1F12A6A6A600000000CB
:104400000001000000000111FFFF00005048593674
:1044100000000000000000000100000015BC0011B9
:104420000B000500F7000000B40000280028002859
:104430003075A000A000A000A00000080008E00166
:10444000F0001000100010001000100010005000CC
:104450005000500010001000D007000000000000C5
:104460000F0001000500307507001000010081FFFA
:1044700000000000FF000000FD7100110570001138
:10448000956D0011FFFF0100FF000000199C001155
:1044900095990011AD980011000000000000000087
:1044A00000000800040000003B0001085902E00180
:1044B00088212800FF0000000200000072BD0011EA
:1044C0000100000038BE0011020000006EBD0011A6
:1044D000010000003545FF1F020000006ABD001109
:1044E000010000008469FF1F020000006EBD001182
:1044F000010000003445FF1F0200000068BD0011EC
:10450000010000003245FF1F020000006EBD0011D7
:10451000010000003045FF1F0200000066BD0011D1
:10452000010000002845FF1F18001800000090013E
:1045300002000003020200000200000072BD001130
:10454000010000004CBE0011020000006EBD001111
:10455000010000007845FF1F0200000064BD00114B
:104560000000000000000000020000006CBD00110F
:0A45700003000000A469FF1F20FFF4
:040000051FFF184180
:00000001FF
